Archive member included because of file (symbol)

c:/pic30_tools/bin/bin/../../lib\libpic30-coff.a(crt1.o)
                              (_resetALT)
c:/pic30_tools/bin/bin/../../lib\libpic30-coff.a(crt0.o)
                              (_resetPRI)
c:/pic30_tools/bin/bin/../../lib\libm-coff.a(divmoddi3.o)
                              ..\Microchip\TCPIP Stack\Objects - COM4201Lab2Solution-C30\Tick.o (__udivdi3)
c:/pic30_tools/bin/bin/../../lib\libm-coff.a(udivsi3.o)
                              ..\Microchip\TCPIP Stack\Objects - COM4201Lab2Solution-C30\Helpers.o (__udivsi3)
c:/pic30_tools/bin/bin/../../lib\libm-coff.a(muldi3.o)
                              ..\Microchip\TCPIP Stack\Objects - COM4201Lab2Solution-C30\TCPPerformanceTest.o (__muldi3)
c:/pic30_tools/bin/bin/../../lib\libm-coff.a(umuldi3.o)
                              c:/pic30_tools/bin/bin/../../lib\libm-coff.a(muldi3.o) (__umuldi3)
c:/pic30_tools/bin/bin/../../lib\libc-coff.a(strlen.o)
                              Objects - COM4201Lab2Solution-C30\MainDemo.o (strlen)
c:/pic30_tools/bin/bin/../../lib\libc-coff.a(memcmp.o)
                              Objects - COM4201Lab2Solution-C30\CustomHTTPApp.o (memcmp)
c:/pic30_tools/bin/bin/../../lib\libc-coff.a(strcmp.o)
                              Objects - COM4201Lab2Solution-C30\CustomHTTPApp.o (strcmp)
c:/pic30_tools/bin/bin/../../lib\libc-coff.a(memset.o)
                              Objects - COM4201Lab2Solution-C30\CustomHTTPApp.o (memset)
c:/pic30_tools/bin/bin/../../lib\libc-coff.a(strcpy.o)
                              Objects - COM4201Lab2Solution-C30\CustomHTTPApp.o (strcpy)
c:/pic30_tools/bin/bin/../../lib\libc-coff.a(xstoul.o)
                              Objects - COM4201Lab2Solution-C30\CustomHTTPApp.o (_Stoul)
c:/pic30_tools/bin/bin/../../lib\libc-coff.a(rand.o)
                              ..\Microchip\TCPIP Stack\Objects - COM4201Lab2Solution-C30\Helpers.o (rand)
c:/pic30_tools/bin/bin/../../lib\libc-coff.a(srand.o)
                              ..\Microchip\TCPIP Stack\Objects - COM4201Lab2Solution-C30\Helpers.o (srand)
c:/pic30_tools/bin/bin/../../lib\libc-coff.a(strchr.o)
                              ..\Microchip\TCPIP Stack\Objects - COM4201Lab2Solution-C30\SMTP.o (strchr)
c:/pic30_tools/bin/bin/../../lib\libc-coff.a(strstr.o)
                              ..\Microchip\TCPIP Stack\Objects - COM4201Lab2Solution-C30\SMTP.o (strstr)
c:/pic30_tools/bin/bin/../../lib\libc-coff.a(memcpy.o)
                              ..\Microchip\TCPIP Stack\Objects - COM4201Lab2Solution-C30\TCP.o (memcpy)
c:/pic30_tools/bin/bin/../../lib\libc-coff.a(isspace.os)
                              c:/pic30_tools/bin/bin/../../lib\libc-coff.a(xstoul.o) (isspace)
c:/pic30_tools/bin/bin/../../lib\libc-coff.a(tolower.os)
                              c:/pic30_tools/bin/bin/../../lib\libc-coff.a(xstoul.o) (tolower)
c:/pic30_tools/bin/bin/../../lib\libc-coff.a(memchr.o)
                              c:/pic30_tools/bin/bin/../../lib\libc-coff.a(xstoul.o) (memchr)
c:/pic30_tools/bin/bin/../../lib\libc-coff.a(errno.o)
                              c:/pic30_tools/bin/bin/../../lib\libc-coff.a(xstoul.o) (errno)
c:/pic30_tools/bin/bin/../../lib\libm-coff.a(mulsi3.o)
                              c:/pic30_tools/bin/bin/../../lib\libc-coff.a(xstoul.o) (__mulsi3)


Program Memory Usage

section                    address   length (PC units)   length (bytes) (dec)
-------                    -------   -----------------   --------------------
.reset                           0                 0x4             0x6  (6)
.ivt                           0x4                0xfc           0x17a  (378)
.aivt                        0x104                0xfc           0x17a  (378)
.text                        0x200               0x650           0x978  (2424)
.const                       0x850              0x1658          0x2184  (8580)
.text                       0x1ea8              0x20ac          0x3102  (12546)
.text                       0x3f54              0x18ee          0x2565  (9573)
.text                       0x5842              0x17dc          0x23ca  (9162)
.text                       0x701e               0xec0          0x1620  (5664)
.text                       0x7ede               0xc2a          0x123f  (4671)
.text                       0x8b08               0xad2          0x103b  (4155)
.text                       0x95da               0x964           0xe16  (3606)
.text                       0x9f3e               0x956           0xe01  (3585)
.text                       0xa894               0x92a           0xdbf  (3519)
.text                       0xb1be               0x8c2           0xd23  (3363)
.text                       0xba80               0x602           0x903  (2307)
.text                       0xc082               0x52e           0x7c5  (1989)
.text                       0xc5b0               0x51a           0x7a7  (1959)
.text                       0xcaca               0x4c4           0x726  (1830)
.text                       0xcf8e               0x434           0x64e  (1614)
.text                       0xd3c2               0x42c           0x642  (1602)
.text                       0xd7ee               0x3a8           0x57c  (1404)
.text                       0xdb96               0x386           0x549  (1353)
.text                       0xdf1c               0x2cc           0x432  (1074)
.text                       0xe1e8               0x2b2           0x40b  (1035)
.dinit                      0xe49a               0x2ac           0x402  (1026)
.text                       0xe746               0x29e           0x3ed  (1005)
.text                       0xe9e4               0x274           0x3ae  (942)
.text                       0xec58               0x262           0x393  (915)
.text                       0xeeba               0x23a           0x357  (855)
.text                       0xf0f4               0x234           0x34e  (846)
.text                       0xf328               0x1e0           0x2d0  (720)
.text                       0xf508               0x1ac           0x282  (642)
.text                       0xf6b4               0x1a8           0x27c  (636)
.text                       0xf85c               0x166           0x219  (537)
.text                       0xf9c2               0x15a           0x207  (519)
.text                       0xfb1c               0x152           0x1fb  (507)
.text                       0xfc6e               0x14e           0x1f5  (501)
.text                       0xfdbc               0x138           0x1d4  (468)
.text                       0xfef4               0x126           0x1b9  (441)
.text                      0x1001a               0x106           0x189  (393)
.text                      0x10120                0xfa           0x177  (375)
.text                      0x1021a                0xdc           0x14a  (330)
.text                      0x102f6                0xd0           0x138  (312)
.text                      0x103c6                0x56            0x81  (129)
.isr                       0x1041c                 0x2             0x3  (3)
__CONFIG2                  0x157fc                 0x2             0x3  (3)
__CONFIG1                  0x157fe                 0x2             0x3  (3)

                     Total program memory used (bytes):        0x1862d  (99885) 75%


Data Memory Usage

section                    address      alignment gaps    total length  (dec)
-------                    -------      --------------    -------------------
TCB_uRAM                     0x800                   0           0x10e  (270)
.nbss                        0x90e                   0           0x160  (352)
HTTP_CONNECTION_STATES       0xa6e                   0            0x8c  (140)
.ndata                       0xafa                   0            0x72  (114)
.nbss                        0xb6c                   0            0xc4  (196)
.ndata                       0xc30                   0            0x50  (80)
.nbss                        0xc80                   0            0x50  (80)
BSD_uRAM                     0xcd0                   0            0x50  (80)
.ndata                       0xd20                   0            0x48  (72)
.nbss                        0xd68                   0            0x80  (128)
SYN_QUEUE_RAM_SECT           0xde8                   0            0x3c  (60)
.nbss                        0xe24                   0            0xe4  (228)
.ndata                       0xf08                   0            0x22  (34)
.nbss                        0xf2a                   0            0xa2  (162)
.ndata                       0xfcc                   0            0x16  (22)
.nbss                        0xfe2                   0            0x44  (68)
.ndata                      0x1026                   0             0xa  (10)
.nbss                       0x1030                   0            0x10  (16)
.ndata                      0x1040                   0             0x6  (6)
.nbss                       0x1046                   0            0x12  (18)
.ndata                      0x1058                   0             0x6  (6)
.nbss                       0x105e                   0             0x4  (4)
.ndata                      0x1062                   0             0x4  (4)
.nbss                       0x1066                   0            0x10  (16)
.ndata                      0x1076                   0             0x8  (8)
_0145ba104acc9c92           0x107e                   0             0x2  (2)
.ndata                      0x1080                   0             0x2  (2)
_01478ee04acc9c98           0x1082                   0             0x2  (2)
.ndata                      0x1084                   0             0x6  (6)
_0148ca804acc9cab           0x108a                   0             0x2  (2)
.ndata                      0x108c                   0             0x6  (6)
.bss                        0x1092                   0            0x88  (136)
.data                       0x111a                   0            0x58  (88)

                        Total data memory used (bytes):          0x972  (2418) 29%


Dynamic Memory Usage

region                     address                      maximum length  (dec)
------                     -------                      ---------------------
heap                             0                                   0  (0)
stack                       0x1172                              0x168e  (5774)

                        Maximum dynamic memory (bytes):         0x168e  (5774)


External Symbols in Data Memory (by address):

                    0x09dc                  _UDPSocketInfo
                    0x0a68                  _activeUDPSocket
                    0x0a6a                  _UDPTxCount
                    0x0a6c                  _UDPRxCount
                    0x0a6e                  _curHTTP
                    0x0af0                  _httpStubs
                    0x0af8                  _curHTTPID
                    0x0bd8                  _lastRead
                    0x0d6c                  _AppConfig
                    0x0d9f                  _AN0String
                    0x0da8                  _lastBlock
                    0x0e4e                  _DDNSClient
                    0x0e80                  _SMTPClient
                    0x0f22                  _ddnsServiceHosts
                    0x0f2a                  _LCDText
                    0x1006                  _remoteNode
                    0x1040                  _smDHCPState
                    0x1042                  _DHCPFlags
                    0x1044                  _DHCPBindCount
                    0x107a                  _myDHCPBindCount
                    0x1080                  _bDHCPServerEnabled
                    0x1164                  __Tls_setup__Randseed
                    0x1166                  __Randseed
                    0x116a                  __Tls_setup__Randinit
                    0x116c                  __Randinit
                    0x116e                  __Tls_setup_errno
                    0x1170                  _errno

External Symbols in Data Memory (by name):

                    0x0d9f                  _AN0String
                    0x0d6c                  _AppConfig
                    0x0e4e                  _DDNSClient
                    0x1044                  _DHCPBindCount
                    0x1042                  _DHCPFlags
                    0x0f2a                  _LCDText
                    0x0e80                  _SMTPClient
                    0x0a6c                  _UDPRxCount
                    0x09dc                  _UDPSocketInfo
                    0x0a6a                  _UDPTxCount
                    0x116c                  __Randinit
                    0x1166                  __Randseed
                    0x116a                  __Tls_setup__Randinit
                    0x1164                  __Tls_setup__Randseed
                    0x116e                  __Tls_setup_errno
                    0x0a68                  _activeUDPSocket
                    0x1080                  _bDHCPServerEnabled
                    0x0a6e                  _curHTTP
                    0x0af8                  _curHTTPID
                    0x0f22                  _ddnsServiceHosts
                    0x1170                  _errno
                    0x0af0                  _httpStubs
                    0x0da8                  _lastBlock
                    0x0bd8                  _lastRead
                    0x107a                  _myDHCPBindCount
                    0x1006                  _remoteNode
                    0x1040                  _smDHCPState

External Symbols in Program Memory (by address):

                  0x000200                  __resetPRI
                  0x00021e                  __psv_init
                  0x00022e                  __data_init
                  0x000288                  _strlen
                  0x000296                  _memcmp
                  0x0002b2                  _strcmp
                  0x0002d6                  _memset
                  0x0002e4                  _strcpy
                  0x0002f4                  __Stoul
                  0x00041c                  _rand
                  0x0004c6                  _srand
                  0x0004e8                  _strchr
                  0x0004fa                  _strstr
                  0x000522                  _memcpy
                  0x000530                  _isspace
                  0x000540                  _tolower
                  0x00054e                  _memchr
                  0x000562                  __Geterrno
                  0x000594                  ___udivmoddi3
                  0x000662                  ___udivdi3
                  0x000670                  ___umoddi3
                  0x000678                  ___divdi3
                  0x0006b2                  ___moddi3
                  0x000784                  ___udivsi3
                  0x0007a4                  ___muldi3
                  0x000800                  ___umuldi3
                  0x000844                  ___mulsi3
                  0x001249                  _HTML_UP_ARROW
                  0x00124c                  _HTML_DOWN_ARROW
                  0x001e08                  _TCPSocketInitializer
                  0x001f5a                  _TCPInit
                  0x00200a                  _TCPOpen
                  0x002150                  _TCPWasReset
                  0x002174                  _TCPIsConnected
                  0x002190                  _TCPDisconnect
                  0x0021fe                  _TCPGetRemoteInfo
                  0x002216                  _TCPFlush
                  0x002232                  _TCPIsPutReady
                  0x00227c                  _TCPPut
                  0x002308                  _TCPPutArray
                  0x0023d6                  _TCPPutString
                  0x0023f4                  _TCPGetTxFIFOFull
                  0x002412                  _TCPDiscard
                  0x002430                  _TCPIsGetReady
                  0x002462                  _TCPGet
                  0x0024cc                  _TCPGetArray
                  0x002588                  _TCPGetRxFIFOFree
                  0x0025a4                  _TCPFindArrayEx
                  0x002828                  _TCPFindEx
                  0x002846                  _TCPTick
                  0x002cb4                  _TCPProcess
                  0x003d3a                  _TCPAdjustFIFOSize
                  0x003f54                  _HTTPNeedsAuth
                  0x003f76                  _HTTPCheckAuth
                  0x003fa4                  _HTTPExecuteGet
                  0x0041ce                  _HTTPExecutePost
                  0x004e2c                  _HTTPPrint_builddate
                  0x004e6c                  _HTTPPrint_version
                  0x004e88                  _HTTPPrint_btn
                  0x004f08                  _HTTPPrint_led
                  0x004fd8                  _HTTPPrint_ledSelected
                  0x0050b2                  _HTTPPrint_pot
                  0x0050d8                  _HTTPPrint_lcdtext
                  0x0051bc                  _HTTPPrint_hellomsg
                  0x0051fa                  _HTTPPrint_cookiename
                  0x00523a                  _HTTPPrint_uploadedmd5
                  0x005314                  _HTTPPrintIP
                  0x005368                  _HTTPPrint_config_hostname
                  0x005382                  _HTTPPrint_config_dhcpchecked
                  0x0053a6                  _HTTPPrint_config_ip
                  0x0053cc                  _HTTPPrint_config_gw
                  0x0053f2                  _HTTPPrint_config_subnet
                  0x005418                  _HTTPPrint_config_dns1
                  0x00543e                  _HTTPPrint_config_dns2
                  0x005464                  _HTTPPrint_config_mac
                  0x005502                  _HTTPPrint_reboot
                  0x00550a                  _HTTPPrint_rebootaddr
                  0x005524                  _HTTPPrint_ddns_user
                  0x00557c                  _HTTPPrint_ddns_pass
                  0x0055d4                  _HTTPPrint_ddns_host
                  0x00562c                  _HTTPPrint_ddns_service
                  0x00566c                  _HTTPPrint_ddns_status
                  0x0056d4                  _HTTPPrint_ddns_status_msg
                  0x0057c6                  _HTTPPrint_status_ok
                  0x005804                  _HTTPPrint_status_fail
                  0x005842                  _HTTPPrint
                  0x005862                  _HTTPPrint_
                  0x00587c                  _HTTPInit
                  0x0058ec                  _HTTPServer
                  0x006a1c                  _HTTPURLDecode
                  0x006ae2                  _HTTPGetArg
                  0x006b2a                  _HTTPReadPostName
                  0x006b52                  _HTTPReadPostValue
                  0x006f56                  _HTTPIncFile
                  0x00701e                  _SMTPBeginUsage
                  0x007072                  _SMTPEndUsage
                  0x0070ba                  _SMTPTask
                  0x007c16                  _SMTPSendMail
                  0x007c1e                  _SMTPIsBusy
                  0x007c34                  _SMTPIsPutReady
                  0x007c50                  _SMTPPut
                  0x007cf0                  _SMTPPutArray
                  0x007d2c                  _SMTPPutString
                  0x007d62                  _SMTPFlush
                  0x007d6e                  _SMTPPutDone
                  0x007ede                  _MACInit
                  0x008002                  _MACIsLinked
                  0x008016                  _MACIsTxReady
                  0x00802e                  _MACDiscardRx
                  0x008062                  _MACGetFreeRxSize
                  0x0080ea                  _MACGetHeader
                  0x0081cc                  _MACPutHeader
                  0x008220                  _MACFlush
                  0x00833c                  _MACSetReadPtrInRx
                  0x00836a                  _MACSetWritePtr
                  0x008398                  _MACSetReadPtr
                  0x0083c6                  _MACCalcRxChecksum
                  0x00841e                  _CalcIPBufferChecksum
                  0x0084d2                  _MACMemCopyAsync
                  0x008680                  _MACIsMemCopyDone
                  0x008698                  _MACGet
                  0x0086c2                  _MACGetArray
                  0x00878a                  _MACPut
                  0x0087bc                  _MACPutArray
                  0x008932                  _ReadPHYReg
                  0x008a3a                  _WritePHYReg
                  0x008a8a                  _MACPowerDown
                  0x008ab8                  _MACPowerUp
                  0x008ad8                  _SetCLKOUT
                  0x008aee                  _GetCLKOUT
                  0x008b08                  _MPFSInit
                  0x008b3e                  _MPFSOpen
                  0x008c8c                  _MPFSOpenID
                  0x008d10                  _MPFSClose
                  0x008d32                  _MPFSGet
                  0x008e38                  _MPFSGetArray
                  0x008f4c                  _MPFSGetLong
                  0x008f6c                  _MPFSSeek
                  0x009148                  _MPFSFormat
                  0x0091e2                  _MPFSPutArray
                  0x009286                  _MPFSPutEnd
                  0x0092e2                  _MPFSGetTimestamp
                  0x009330                  _MPFSGetMicrotime
                  0x00937e                  _MPFSGetFlags
                  0x0093c2                  _MPFSGetSize
                  0x009410                  _MPFSGetBytesRem
                  0x009458                  _MPFSGetStartAddr
                  0x0094a8                  _MPFSGetEndAddr
                  0x009502                  _MPFSGetFilename
                  0x00956a                  _MPFSGetPosition
                  0x00958a                  _MPFSGetID
                  0x0095da                  _DDNSInit
                  0x00961c                  _DDNSTask
                  0x009ef4                  _DDNSForceUpdate
                  0x009f0a                  _DDNSSetService
                  0x009f2a                  _DDNSGetLastIP
                  0x009f36                  _DDNSGetLastStatus
                  0x009f3e                  _GenerateRandomDWORD
                  0x00a058                  _StringToIPAddress
                  0x00a1d8                  _Base64Decode
                  0x00a33e                  _Base64Encode
                  0x00a49a                  _uitoa
                  0x00a518                  _ultoa
                  0x00a5c8                  _hexatob
                  0x00a63e                  _btohexa_high
                  0x00a666                  _btohexa_low
                  0x00a68c                  _stricmppgm2ram
                  0x00a724                  _swaps
                  0x00a73e                  _swapl
                  0x00a79c                  _CalcIPChecksum
                  0x00a812                  _strupr
                  0x00a84c                  _FormatNetBIOSName
                  0x00a894                  _BerkeleySocketInit
                  0x00a8d6                  _socket
                  0x00a954                  _bind
                  0x00a9c8                  _listen
                  0x00aa14                  _accept
                  0x00ab40                  _connect
                  0x00ac7e                  _send
                  0x00adc0                  _sendto
                  0x00af02                  _recv
                  0x00b04c                  _recvfrom
                  0x00b106                  _gethostname
                  0x00b16a                  _closesocket
                  0x00b1be                  _DHCPReset
                  0x00b1e0                  _DHCPDisable
                  0x00b1fc                  _DHCPEnable
                  0x00b214                  _DHCPTask
                  0x00ba80                  _DNSBeginUsage
                  0x00ba9c                  _DNSEndUsage
                  0x00bac2                  _DNSResolve
                  0x00baf2                  _DNSIsResolved
                  0x00c082                  _UDPInit
                  0x00c09c                  _UDPTask
                  0x00c0a6                  _UDPOpen
                  0x00c134                  _UDPClose
                  0x00c15e                  _UDPSetTxBuffer
                  0x00c172                  _UDPSetRxBuffer
                  0x00c186                  _UDPIsPutReady
                  0x00c1bc                  _UDPPut
                  0x00c1f0                  _UDPPutArray
                  0x00c228                  _UDPPutString
                  0x00c23e                  _UDPFlush
                  0x00c314                  _UDPIsGetReady
                  0x00c340                  _UDPGet
                  0x00c376                  _UDPGetArray
                  0x00c3c0                  _UDPDiscard
                  0x00c3d8                  _UDPProcess
                  0x00c5b0                  _DHCPServerTask
                  0x00caca                  _HashAddData
                  0x00cae6                  _MD5Initialize
                  0x00cb22                  _MD5AddData
                  0x00ce22                  _MD5Calculate
                  0x00cf8e                  __AddressError
                  0x00cf98                  __StackError
                  0x00cfa2                  _main
                  0x00d0e2                  _DisplayIPValue
                  0x00d38a                  _SaveAppConfig
                  0x00d3c2                  _TelnetTask
                  0x00d868                  _ARPInit
                  0x00d89e                  _ARPProcess
                  0x00d99e                  _ARPResolve
                  0x00da6a                  _ARPIsResolved
                  0x00db96                  _NBNSTask
                  0x00df1c                  _SNTPClient
                  0x00e190                  _SNTPGetUTCSeconds
                  0x00e1e8                  _TCPPerformanceTask
                  0x00e1f2                  _TCPTXPerformanceTask
                  0x00e388                  _TCPRXPerformanceTask
                  0x00e746                  _BerkeleyUDPClientDemo
                  0x00e98c                  _BerkeleySNTPGetUTCSeconds
                  0x00e9e4                  _StackInit
                  0x00ea20                  _StackTask
                  0x00ec26                  _StackApplications
                  0x00ec58                  _DoUARTConfig
                  0x00eeba                  _XEEInit
                  0x00eed8                  _XEEBeginRead
                  0x00eeec                  _XEERead
                  0x00ef20                  _XEEEndRead
                  0x00ef28                  _XEEReadArray
                  0x00efb6                  _XEEBeginWrite
                  0x00efca                  _XEEWrite
                  0x00efe6                  _XEEEndWrite
                  0x00f0b4                  _XEEIsBusy
                  0x00f0f4                  _ICMPProcess
                  0x00f1b6                  _ICMPSendPing
                  0x00f234                  _ICMPGetReply
                  0x00f304                  _ICMPBeginUsage
                  0x00f320                  _ICMPEndUsage
                  0x00f328                  _UART2TCPBridgeInit
                  0x00f33e                  _UART2TCPBridgeTask
                  0x00f49a                  __U2RXInterrupt
                  0x00f4d8                  __U2TXInterrupt
                  0x00f508                  _IPGetHeader
                  0x00f5d2                  _IPPutHeader
                  0x00f670                  _IPSetRxBuffer
                  0x00f6f8                  _LCDInit
                  0x00f784                  _LCDUpdate
                  0x00f840                  _LCDErase
                  0x00f85c                  _AnnounceIP
                  0x00f8de                  _DiscoveryTask
                  0x00f9c2                  _GenericTCPClient
                  0x00fb1c                  _ReadStringUART
                  0x00fb64                  _putsUART2
                  0x00fbb2                  _getsUART2
                  0x00fc1a                  _DataRdyUART2
                  0x00fc26                  _BusyUART2
                  0x00fc34                  _ReadUART2
                  0x00fc52                  _WriteUART2
                  0x00fc6e                  _RebootTask
                  0x00fdbc                  _BerkeleyTCPServerDemo
                  0x00fef4                  _BerkeleyTCPClientDemo
                  0x01001a                  _SMTPDemo
                  0x010120                  _TickInit
                  0x01019c                  _TickGet
                  0x0101a8                  _TickGetDiv256
                  0x0101c2                  _TickGetDiv64K
                  0x0101dc                  _TickConvertToMilliseconds
                  0x010202                  __T1Interrupt
                  0x01021a                  _PingDemo
                  0x0102f6                  _GenericTCPServer
                  0x0103c6                  _DelayMs
                  0x0103f0                  _Delay10us
                  0x01041c                  __DefaultInterrupt

External Symbols in Program Memory (by name):

                  0x00d868                  _ARPInit
                  0x00da6a                  _ARPIsResolved
                  0x00d89e                  _ARPProcess
                  0x00d99e                  _ARPResolve
                  0x00f85c                  _AnnounceIP
                  0x00a1d8                  _Base64Decode
                  0x00a33e                  _Base64Encode
                  0x00e98c                  _BerkeleySNTPGetUTCSeconds
                  0x00a894                  _BerkeleySocketInit
                  0x00fef4                  _BerkeleyTCPClientDemo
                  0x00fdbc                  _BerkeleyTCPServerDemo
                  0x00e746                  _BerkeleyUDPClientDemo
                  0x00fc26                  _BusyUART2
                  0x00841e                  _CalcIPBufferChecksum
                  0x00a79c                  _CalcIPChecksum
                  0x009ef4                  _DDNSForceUpdate
                  0x009f2a                  _DDNSGetLastIP
                  0x009f36                  _DDNSGetLastStatus
                  0x0095da                  _DDNSInit
                  0x009f0a                  _DDNSSetService
                  0x00961c                  _DDNSTask
                  0x00b1e0                  _DHCPDisable
                  0x00b1fc                  _DHCPEnable
                  0x00b1be                  _DHCPReset
                  0x00c5b0                  _DHCPServerTask
                  0x00b214                  _DHCPTask
                  0x00ba80                  _DNSBeginUsage
                  0x00ba9c                  _DNSEndUsage
                  0x00baf2                  _DNSIsResolved
                  0x00bac2                  _DNSResolve
                  0x00fc1a                  _DataRdyUART2
                  0x0103f0                  _Delay10us
                  0x0103c6                  _DelayMs
                  0x00f8de                  _DiscoveryTask
                  0x00d0e2                  _DisplayIPValue
                  0x00ec58                  _DoUARTConfig
                  0x00a84c                  _FormatNetBIOSName
                  0x009f3e                  _GenerateRandomDWORD
                  0x00f9c2                  _GenericTCPClient
                  0x0102f6                  _GenericTCPServer
                  0x008aee                  _GetCLKOUT
                  0x00124c                  _HTML_DOWN_ARROW
                  0x001249                  _HTML_UP_ARROW
                  0x003f76                  _HTTPCheckAuth
                  0x003fa4                  _HTTPExecuteGet
                  0x0041ce                  _HTTPExecutePost
                  0x006ae2                  _HTTPGetArg
                  0x006f56                  _HTTPIncFile
                  0x00587c                  _HTTPInit
                  0x003f54                  _HTTPNeedsAuth
                  0x005842                  _HTTPPrint
                  0x005314                  _HTTPPrintIP
                  0x005862                  _HTTPPrint_
                  0x004e88                  _HTTPPrint_btn
                  0x004e2c                  _HTTPPrint_builddate
                  0x005382                  _HTTPPrint_config_dhcpchecked
                  0x005418                  _HTTPPrint_config_dns1
                  0x00543e                  _HTTPPrint_config_dns2
                  0x0053cc                  _HTTPPrint_config_gw
                  0x005368                  _HTTPPrint_config_hostname
                  0x0053a6                  _HTTPPrint_config_ip
                  0x005464                  _HTTPPrint_config_mac
                  0x0053f2                  _HTTPPrint_config_subnet
                  0x0051fa                  _HTTPPrint_cookiename
                  0x0055d4                  _HTTPPrint_ddns_host
                  0x00557c                  _HTTPPrint_ddns_pass
                  0x00562c                  _HTTPPrint_ddns_service
                  0x00566c                  _HTTPPrint_ddns_status
                  0x0056d4                  _HTTPPrint_ddns_status_msg
                  0x005524                  _HTTPPrint_ddns_user
                  0x0051bc                  _HTTPPrint_hellomsg
                  0x0050d8                  _HTTPPrint_lcdtext
                  0x004f08                  _HTTPPrint_led
                  0x004fd8                  _HTTPPrint_ledSelected
                  0x0050b2                  _HTTPPrint_pot
                  0x005502                  _HTTPPrint_reboot
                  0x00550a                  _HTTPPrint_rebootaddr
                  0x005804                  _HTTPPrint_status_fail
                  0x0057c6                  _HTTPPrint_status_ok
                  0x00523a                  _HTTPPrint_uploadedmd5
                  0x004e6c                  _HTTPPrint_version
                  0x006b2a                  _HTTPReadPostName
                  0x006b52                  _HTTPReadPostValue
                  0x0058ec                  _HTTPServer
                  0x006a1c                  _HTTPURLDecode
                  0x00caca                  _HashAddData
                  0x00f304                  _ICMPBeginUsage
                  0x00f320                  _ICMPEndUsage
                  0x00f234                  _ICMPGetReply
                  0x00f0f4                  _ICMPProcess
                  0x00f1b6                  _ICMPSendPing
                  0x00f508                  _IPGetHeader
                  0x00f5d2                  _IPPutHeader
                  0x00f670                  _IPSetRxBuffer
                  0x00f840                  _LCDErase
                  0x00f6f8                  _LCDInit
                  0x00f784                  _LCDUpdate
                  0x0083c6                  _MACCalcRxChecksum
                  0x00802e                  _MACDiscardRx
                  0x008220                  _MACFlush
                  0x008698                  _MACGet
                  0x0086c2                  _MACGetArray
                  0x008062                  _MACGetFreeRxSize
                  0x0080ea                  _MACGetHeader
                  0x007ede                  _MACInit
                  0x008002                  _MACIsLinked
                  0x008680                  _MACIsMemCopyDone
                  0x008016                  _MACIsTxReady
                  0x0084d2                  _MACMemCopyAsync
                  0x008a8a                  _MACPowerDown
                  0x008ab8                  _MACPowerUp
                  0x00878a                  _MACPut
                  0x0087bc                  _MACPutArray
                  0x0081cc                  _MACPutHeader
                  0x008398                  _MACSetReadPtr
                  0x00833c                  _MACSetReadPtrInRx
                  0x00836a                  _MACSetWritePtr
                  0x00cb22                  _MD5AddData
                  0x00ce22                  _MD5Calculate
                  0x00cae6                  _MD5Initialize
                  0x008d10                  _MPFSClose
                  0x009148                  _MPFSFormat
                  0x008d32                  _MPFSGet
                  0x008e38                  _MPFSGetArray
                  0x009410                  _MPFSGetBytesRem
                  0x0094a8                  _MPFSGetEndAddr
                  0x009502                  _MPFSGetFilename
                  0x00937e                  _MPFSGetFlags
                  0x00958a                  _MPFSGetID
                  0x008f4c                  _MPFSGetLong
                  0x009330                  _MPFSGetMicrotime
                  0x00956a                  _MPFSGetPosition
                  0x0093c2                  _MPFSGetSize
                  0x009458                  _MPFSGetStartAddr
                  0x0092e2                  _MPFSGetTimestamp
                  0x008b08                  _MPFSInit
                  0x008b3e                  _MPFSOpen
                  0x008c8c                  _MPFSOpenID
                  0x0091e2                  _MPFSPutArray
                  0x009286                  _MPFSPutEnd
                  0x008f6c                  _MPFSSeek
                  0x00db96                  _NBNSTask
                  0x01021a                  _PingDemo
                  0x008932                  _ReadPHYReg
                  0x00fb1c                  _ReadStringUART
                  0x00fc34                  _ReadUART2
                  0x00fc6e                  _RebootTask
                  0x00701e                  _SMTPBeginUsage
                  0x01001a                  _SMTPDemo
                  0x007072                  _SMTPEndUsage
                  0x007d62                  _SMTPFlush
                  0x007c1e                  _SMTPIsBusy
                  0x007c34                  _SMTPIsPutReady
                  0x007c50                  _SMTPPut
                  0x007cf0                  _SMTPPutArray
                  0x007d6e                  _SMTPPutDone
                  0x007d2c                  _SMTPPutString
                  0x007c16                  _SMTPSendMail
                  0x0070ba                  _SMTPTask
                  0x00df1c                  _SNTPClient
                  0x00e190                  _SNTPGetUTCSeconds
                  0x00d38a                  _SaveAppConfig
                  0x008ad8                  _SetCLKOUT
                  0x00ec26                  _StackApplications
                  0x00e9e4                  _StackInit
                  0x00ea20                  _StackTask
                  0x00a058                  _StringToIPAddress
                  0x003d3a                  _TCPAdjustFIFOSize
                  0x002412                  _TCPDiscard
                  0x002190                  _TCPDisconnect
                  0x0025a4                  _TCPFindArrayEx
                  0x002828                  _TCPFindEx
                  0x002216                  _TCPFlush
                  0x002462                  _TCPGet
                  0x0024cc                  _TCPGetArray
                  0x0021fe                  _TCPGetRemoteInfo
                  0x002588                  _TCPGetRxFIFOFree
                  0x0023f4                  _TCPGetTxFIFOFull
                  0x001f5a                  _TCPInit
                  0x002174                  _TCPIsConnected
                  0x002430                  _TCPIsGetReady
                  0x002232                  _TCPIsPutReady
                  0x00200a                  _TCPOpen
                  0x00e1e8                  _TCPPerformanceTask
                  0x002cb4                  _TCPProcess
                  0x00227c                  _TCPPut
                  0x002308                  _TCPPutArray
                  0x0023d6                  _TCPPutString
                  0x00e388                  _TCPRXPerformanceTask
                  0x001e08                  _TCPSocketInitializer
                  0x00e1f2                  _TCPTXPerformanceTask
                  0x002846                  _TCPTick
                  0x002150                  _TCPWasReset
                  0x00d3c2                  _TelnetTask
                  0x0101dc                  _TickConvertToMilliseconds
                  0x01019c                  _TickGet
                  0x0101a8                  _TickGetDiv256
                  0x0101c2                  _TickGetDiv64K
                  0x010120                  _TickInit
                  0x00f328                  _UART2TCPBridgeInit
                  0x00f33e                  _UART2TCPBridgeTask
                  0x00c134                  _UDPClose
                  0x00c3c0                  _UDPDiscard
                  0x00c23e                  _UDPFlush
                  0x00c340                  _UDPGet
                  0x00c376                  _UDPGetArray
                  0x00c082                  _UDPInit
                  0x00c314                  _UDPIsGetReady
                  0x00c186                  _UDPIsPutReady
                  0x00c0a6                  _UDPOpen
                  0x00c3d8                  _UDPProcess
                  0x00c1bc                  _UDPPut
                  0x00c1f0                  _UDPPutArray
                  0x00c228                  _UDPPutString
                  0x00c172                  _UDPSetRxBuffer
                  0x00c15e                  _UDPSetTxBuffer
                  0x00c09c                  _UDPTask
                  0x008a3a                  _WritePHYReg
                  0x00fc52                  _WriteUART2
                  0x00eed8                  _XEEBeginRead
                  0x00efb6                  _XEEBeginWrite
                  0x00ef20                  _XEEEndRead
                  0x00efe6                  _XEEEndWrite
                  0x00eeba                  _XEEInit
                  0x00f0b4                  _XEEIsBusy
                  0x00eeec                  _XEERead
                  0x00ef28                  _XEEReadArray
                  0x00efca                  _XEEWrite
                  0x00cf8e                  __AddressError
                  0x01041c                  __DefaultInterrupt
                  0x000562                  __Geterrno
                  0x00cf98                  __StackError
                  0x0002f4                  __Stoul
                  0x010202                  __T1Interrupt
                  0x00f49a                  __U2RXInterrupt
                  0x00f4d8                  __U2TXInterrupt
                  0x000678                  ___divdi3
                  0x0006b2                  ___moddi3
                  0x0007a4                  ___muldi3
                  0x000844                  ___mulsi3
                  0x000662                  ___udivdi3
                  0x000594                  ___udivmoddi3
                  0x000784                  ___udivsi3
                  0x000670                  ___umoddi3
                  0x000800                  ___umuldi3
                  0x00022e                  __data_init
                  0x00021e                  __psv_init
                  0x000200                  __resetPRI
                  0x00aa14                  _accept
                  0x00a954                  _bind
                  0x00a63e                  _btohexa_high
                  0x00a666                  _btohexa_low
                  0x00b16a                  _closesocket
                  0x00ab40                  _connect
                  0x00b106                  _gethostname
                  0x00fbb2                  _getsUART2
                  0x00a5c8                  _hexatob
                  0x000530                  _isspace
                  0x00a9c8                  _listen
                  0x00cfa2                  _main
                  0x00054e                  _memchr
                  0x000296                  _memcmp
                  0x000522                  _memcpy
                  0x0002d6                  _memset
                  0x00fb64                  _putsUART2
                  0x00041c                  _rand
                  0x00af02                  _recv
                  0x00b04c                  _recvfrom
                  0x00ac7e                  _send
                  0x00adc0                  _sendto
                  0x00a8d6                  _socket
                  0x0004c6                  _srand
                  0x0004e8                  _strchr
                  0x0002b2                  _strcmp
                  0x0002e4                  _strcpy
                  0x00a68c                  _stricmppgm2ram
                  0x000288                  _strlen
                  0x0004fa                  _strstr
                  0x00a812                  _strupr
                  0x00a73e                  _swapl
                  0x00a724                  _swaps
                  0x000540                  _tolower
                  0x00a49a                  _uitoa
                  0x00a518                  _ultoa

Memory Configuration

Name             Origin             Length             Attributes
data             0x000800           0x002000           a !xr
reset            0x000000           0x000004  
ivt              0x000004           0x0000fc  
aivt             0x000104           0x0000fc  
program          0x000200           0x0155fc           xr
config2          0x0157fc           0x000002  
config1          0x0157fe           0x000002  
*default*        0x000000           0xffffffff  

Linker script and memory map

LOAD Objects - COM4201Lab2Solution-C30\MainDemo.o
LOAD Objects - COM4201Lab2Solution-C30\CustomHTTPApp.o
LOAD ..\Microchip\TCPIP Stack\Objects - COM4201Lab2Solution-C30\Tick.o
LOAD ..\Microchip\TCPIP Stack\Objects - COM4201Lab2Solution-C30\UART2TCPBridge.o
LOAD ..\Microchip\TCPIP Stack\Objects - COM4201Lab2Solution-C30\UART.o
LOAD ..\Microchip\TCPIP Stack\Objects - COM4201Lab2Solution-C30\UDP.o
LOAD ..\Microchip\TCPIP Stack\Objects - COM4201Lab2Solution-C30\UDPPerformanceTest.o
LOAD ..\Microchip\TCPIP Stack\Objects - COM4201Lab2Solution-C30\Announce.o
LOAD ..\Microchip\TCPIP Stack\Objects - COM4201Lab2Solution-C30\ARP.o
LOAD ..\Microchip\TCPIP Stack\Objects - COM4201Lab2Solution-C30\Delay.o
LOAD ..\Microchip\TCPIP Stack\Objects - COM4201Lab2Solution-C30\DHCP.o
LOAD ..\Microchip\TCPIP Stack\Objects - COM4201Lab2Solution-C30\DHCPs.o
LOAD ..\Microchip\TCPIP Stack\Objects - COM4201Lab2Solution-C30\DNS.o
LOAD ..\Microchip\TCPIP Stack\Objects - COM4201Lab2Solution-C30\DynDNS.o
LOAD ..\Microchip\TCPIP Stack\Objects - COM4201Lab2Solution-C30\ENC28J60.o
LOAD ..\Microchip\TCPIP Stack\Objects - COM4201Lab2Solution-C30\ETH97J60.o
LOAD ..\Microchip\TCPIP Stack\Objects - COM4201Lab2Solution-C30\FTP.o
LOAD ..\Microchip\TCPIP Stack\Objects - COM4201Lab2Solution-C30\Hashes.o
LOAD ..\Microchip\TCPIP Stack\Objects - COM4201Lab2Solution-C30\Helpers.o
LOAD ..\Microchip\TCPIP Stack\Objects - COM4201Lab2Solution-C30\HTTP2.o
LOAD ..\Microchip\TCPIP Stack\Objects - COM4201Lab2Solution-C30\HTTP.o
LOAD ..\Microchip\TCPIP Stack\Objects - COM4201Lab2Solution-C30\ICMP.o
LOAD ..\Microchip\TCPIP Stack\Objects - COM4201Lab2Solution-C30\IP.o
LOAD ..\Microchip\TCPIP Stack\Objects - COM4201Lab2Solution-C30\LCDBlocking.o
LOAD ..\Microchip\TCPIP Stack\Objects - COM4201Lab2Solution-C30\MPFS2.o
LOAD ..\Microchip\TCPIP Stack\Objects - COM4201Lab2Solution-C30\MPFS.o
LOAD ..\Microchip\TCPIP Stack\Objects - COM4201Lab2Solution-C30\NBNS.o
LOAD ..\Microchip\TCPIP Stack\Objects - COM4201Lab2Solution-C30\Reboot.o
LOAD ..\Microchip\TCPIP Stack\Objects - COM4201Lab2Solution-C30\SMTP.o
LOAD ..\Microchip\TCPIP Stack\Objects - COM4201Lab2Solution-C30\SNMP.o
LOAD ..\Microchip\TCPIP Stack\Objects - COM4201Lab2Solution-C30\SNTP.o
LOAD ..\Microchip\TCPIP Stack\Objects - COM4201Lab2Solution-C30\SPIEEPROM.o
LOAD ..\Microchip\TCPIP Stack\Objects - COM4201Lab2Solution-C30\SPIFlash.o
LOAD ..\Microchip\TCPIP Stack\Objects - COM4201Lab2Solution-C30\SPIRAM.o
LOAD ..\Microchip\TCPIP Stack\Objects - COM4201Lab2Solution-C30\StackTsk.o
LOAD ..\Microchip\TCPIP Stack\Objects - COM4201Lab2Solution-C30\TCP.o
LOAD ..\Microchip\TCPIP Stack\Objects - COM4201Lab2Solution-C30\TCPPerformanceTest.o
LOAD ..\Microchip\TCPIP Stack\Objects - COM4201Lab2Solution-C30\Telnet.o
LOAD ..\Microchip\TCPIP Stack\Objects - COM4201Lab2Solution-C30\TFTPc.o
LOAD Objects - COM4201Lab2Solution-C30\CustomSNMPApp.o
LOAD Objects - COM4201Lab2Solution-C30\UARTConfig.o
LOAD Objects - COM4201Lab2Solution-C30\GenericTCPClient.o
LOAD Objects - COM4201Lab2Solution-C30\GenericTCPServer.o
LOAD Objects - COM4201Lab2Solution-C30\PingDemo.o
LOAD Objects - COM4201Lab2Solution-C30\SMTPDemo.o
LOAD Objects - COM4201Lab2Solution-C30\LegacyHTTPApp.o
LOAD ..\Microchip\TCPIP Stack\Objects - COM4201Lab2Solution-C30\BerkeleyAPI.o
LOAD Objects - COM4201Lab2Solution-C30\BerkeleyUDPClientDemo.o
LOAD Objects - COM4201Lab2Solution-C30\BerkeleyTCPClientDemo.o
LOAD Objects - COM4201Lab2Solution-C30\BerkeleyTCPServerDemo.o
LOAD c:/pic30_tools/bin/bin/../../lib/PIC24F\libpPIC24Fxxx-coff.a
                    0x157fc                  __CONFIG2 = 0x157fc
                    0x157fe                  __CONFIG1 = 0x157fe
                    0x0004                  __IVT_BASE = 0x4
                    0x0104                  __AIVT_BASE = 0x104
                    0x0800                  __DATA_BASE = 0x800
                    0x0200                  __CODE_BASE = 0x200

.reset            0x000000          0x4
                  0x000000          0x2 SHORT 0x200 <code 337> (__reset)
                  0x000001          0x2 SHORT 0x4
                  0x000002          0x2 SHORT 0x0 ((<code 337> (__reset) >> 0x10) & 0x7f)
                  0x000003          0x2 SHORT 0x0

.text             0x000200        0x650
 *(.init)
 .init            0x000200         0x88 c:/pic30_tools/bin/bin/../../lib\libpic30-coff.a(crt0.o)
                  0x000200                  _resetPRI
                  0x000200                  _reset
                  0x00021e                  _psv_init
                  0x00022e                  _data_init
 *(.user_init)
 *(.handle)
 *(.libc)
 .libc            0x000288          0xe c:/pic30_tools/bin/bin/../../lib\libc-coff.a(strlen.o)
                  0x000288                  strlen
 .libc            0x000296         0x1c c:/pic30_tools/bin/bin/../../lib\libc-coff.a(memcmp.o)
                  0x000296                  memcmp
 .libc            0x0002b2         0x24 c:/pic30_tools/bin/bin/../../lib\libc-coff.a(strcmp.o)
                  0x0002b2                  strcmp
 .libc            0x0002d6          0xe c:/pic30_tools/bin/bin/../../lib\libc-coff.a(memset.o)
                  0x0002d6                  memset
 .libc            0x0002e4         0x10 c:/pic30_tools/bin/bin/../../lib\libc-coff.a(strcpy.o)
                  0x0002e4                  strcpy
 .libc            0x0002f4        0x128 c:/pic30_tools/bin/bin/../../lib\libc-coff.a(xstoul.o)
                  0x0002f4                  _Stoul
 .libc            0x00041c         0xaa c:/pic30_tools/bin/bin/../../lib\libc-coff.a(rand.o)
                  0x00041c                  rand
 .libc            0x0004c6         0x22 c:/pic30_tools/bin/bin/../../lib\libc-coff.a(srand.o)
                  0x0004c6                  srand
 .libc            0x0004e8         0x12 c:/pic30_tools/bin/bin/../../lib\libc-coff.a(strchr.o)
                  0x0004e8                  strchr
 .libc            0x0004fa         0x28 c:/pic30_tools/bin/bin/../../lib\libc-coff.a(strstr.o)
                  0x0004fa                  strstr
 .libc            0x000522          0xe c:/pic30_tools/bin/bin/../../lib\libc-coff.a(memcpy.o)
                  0x000522                  memcpy
 .libc            0x000530         0x10 c:/pic30_tools/bin/bin/../../lib\libc-coff.a(isspace.os)
                  0x000530                  isspace
 .libc            0x000540          0xe c:/pic30_tools/bin/bin/../../lib\libc-coff.a(tolower.os)
                  0x000540                  tolower
 .libc            0x00054e         0x14 c:/pic30_tools/bin/bin/../../lib\libc-coff.a(memchr.o)
                  0x00054e                  memchr
 .libc            0x000562          0xc c:/pic30_tools/bin/bin/../../lib\libc-coff.a(errno.o)
                  0x000562                  _Geterrno
 *(.libm)
 .libm            0x00056e        0x216 c:/pic30_tools/bin/bin/../../lib\libm-coff.a(divmoddi3.o)
                  0x000594                  __udivmoddi3
                  0x000662                  __udivdi3
                  0x000670                  __umoddi3
                  0x000678                  __divdi3
                  0x0006b2                  __moddi3
 .libm            0x000784         0x20 c:/pic30_tools/bin/bin/../../lib\libm-coff.a(udivsi3.o)
                  0x000784                  __udivsi3
 .libm            0x0007a4         0x5c c:/pic30_tools/bin/bin/../../lib\libm-coff.a(muldi3.o)
                  0x0007a4                  __muldi3
 .libm            0x000800         0x44 c:/pic30_tools/bin/bin/../../lib\libm-coff.a(umuldi3.o)
                  0x000800                  __umuldi3
 .libm            0x000844          0xc c:/pic30_tools/bin/bin/../../lib\libm-coff.a(mulsi3.o)
                  0x000844                  __mulsi3
 *(.libdsp)
 *(.lib*)

__CONFIG2         0x0157fc          0x2
 *(__CONFIG2.sec)
 __CONFIG2.sec    0x0157fc          0x2 Objects - COM4201Lab2Solution-C30\MainDemo.o

__CONFIG1         0x0157fe          0x2
 *(__CONFIG1.sec)
 __CONFIG1.sec    0x0157fe          0x2 Objects - COM4201Lab2Solution-C30\MainDemo.o

.comment
 *(.comment)

.debug_info
 *(.debug_info)
 *(.gnu.linkonce.wi.*)

.debug_abbrev
 *(.debug_abbrev)

.debug_line
 *(.debug_line)

.debug_frame
 *(.debug_frame)

.debug_str
 *(.debug_str)

.debug_loc
 *(.debug_loc)

.debug_macinfo
 *(.debug_macinfo)

.debug_pubnames
 *(.debug_pubnames)

.debug_ranges
 *(.debug_ranges)

.debug_aranges
 *(.debug_aranges)

.ivt              0x000004         0xfc
                  0x000004          0x4 LONG 0x1041c DEFINED (__ReservedTrap0)?<code 337> (__ReservedTrap0):<code 337> (__DefaultInterrupt)
                  0x000006          0x4 LONG 0x1041c DEFINED (__OscillatorFail)?<code 337> (__OscillatorFail):<code 337> (__DefaultInterrupt)
                  0x000008          0x4 LONG 0xcf8e DEFINED (__AddressError)?<code 337> (__AddressError):<code 337> (__DefaultInterrupt)
                  0x00000a          0x4 LONG 0xcf98 DEFINED (__StackError)?<code 337> (__StackError):<code 337> (__DefaultInterrupt)
                  0x00000c          0x4 LONG 0x1041c DEFINED (__MathError)?<code 337> (__MathError):<code 337> (__DefaultInterrupt)
                  0x00000e          0x4 LONG 0x1041c DEFINED (__ReservedTrap5)?<code 337> (__ReservedTrap5):<code 337> (__DefaultInterrupt)
                  0x000010          0x4 LONG 0x1041c DEFINED (__ReservedTrap6)?<code 337> (__ReservedTrap6):<code 337> (__DefaultInterrupt)
                  0x000012          0x4 LONG 0x1041c DEFINED (__ReservedTrap7)?<code 337> (__ReservedTrap7):<code 337> (__DefaultInterrupt)
                  0x000014          0x4 LONG 0x1041c DEFINED (__INT0Interrupt)?<code 337> (__INT0Interrupt):<code 337> (__DefaultInterrupt)
                  0x000016          0x4 LONG 0x1041c DEFINED (__IC1Interrupt)?<code 337> (__IC1Interrupt):<code 337> (__DefaultInterrupt)
                  0x000018          0x4 LONG 0x1041c DEFINED (__OC1Interrupt)?<code 337> (__OC1Interrupt):<code 337> (__DefaultInterrupt)
                  0x00001a          0x4 LONG 0x10202 DEFINED (__T1Interrupt)?<code 337> (__T1Interrupt):<code 337> (__DefaultInterrupt)
                  0x00001c          0x4 LONG 0x1041c DEFINED (__Interrupt4)?<code 337> (__Interrupt4):<code 337> (__DefaultInterrupt)
                  0x00001e          0x4 LONG 0x1041c DEFINED (__IC2Interrupt)?<code 337> (__IC2Interrupt):<code 337> (__DefaultInterrupt)
                  0x000020          0x4 LONG 0x1041c DEFINED (__OC2Interrupt)?<code 337> (__OC2Interrupt):<code 337> (__DefaultInterrupt)
                  0x000022          0x4 LONG 0x1041c DEFINED (__T2Interrupt)?<code 337> (__T2Interrupt):<code 337> (__DefaultInterrupt)
                  0x000024          0x4 LONG 0x1041c DEFINED (__T3Interrupt)?<code 337> (__T3Interrupt):<code 337> (__DefaultInterrupt)
                  0x000026          0x4 LONG 0x1041c DEFINED (__SPI1ErrInterrupt)?<code 337> (__SPI1ErrInterrupt):<code 337> (__DefaultInterrupt)
                  0x000028          0x4 LONG 0x1041c DEFINED (__SPI1Interrupt)?<code 337> (__SPI1Interrupt):<code 337> (__DefaultInterrupt)
                  0x00002a          0x4 LONG 0x1041c DEFINED (__U1RXInterrupt)?<code 337> (__U1RXInterrupt):<code 337> (__DefaultInterrupt)
                  0x00002c          0x4 LONG 0x1041c DEFINED (__U1TXInterrupt)?<code 337> (__U1TXInterrupt):<code 337> (__DefaultInterrupt)
                  0x00002e          0x4 LONG 0x1041c DEFINED (__ADC1Interrupt)?<code 337> (__ADC1Interrupt):<code 337> (__DefaultInterrupt)
                  0x000030          0x4 LONG 0x1041c DEFINED (__Interrupt14)?<code 337> (__Interrupt14):<code 337> (__DefaultInterrupt)
                  0x000032          0x4 LONG 0x1041c DEFINED (__Interrupt15)?<code 337> (__Interrupt15):<code 337> (__DefaultInterrupt)
                  0x000034          0x4 LONG 0x1041c DEFINED (__SI2C1Interrupt)?<code 337> (__SI2C1Interrupt):<code 337> (__DefaultInterrupt)
                  0x000036          0x4 LONG 0x1041c DEFINED (__MI2C1Interrupt)?<code 337> (__MI2C1Interrupt):<code 337> (__DefaultInterrupt)
                  0x000038          0x4 LONG 0x1041c DEFINED (__CompInterrupt)?<code 337> (__CompInterrupt):<code 337> (__DefaultInterrupt)
                  0x00003a          0x4 LONG 0x1041c DEFINED (__CNInterrupt)?<code 337> (__CNInterrupt):<code 337> (__DefaultInterrupt)
                  0x00003c          0x4 LONG 0x1041c DEFINED (__INT1Interrupt)?<code 337> (__INT1Interrupt):<code 337> (__DefaultInterrupt)
                  0x00003e          0x4 LONG 0x1041c DEFINED (__Interrupt21)?<code 337> (__Interrupt21):<code 337> (__DefaultInterrupt)
                  0x000040          0x4 LONG 0x1041c DEFINED (__Interrupt22)?<code 337> (__Interrupt22):<code 337> (__DefaultInterrupt)
                  0x000042          0x4 LONG 0x1041c DEFINED (__Interrupt23)?<code 337> (__Interrupt23):<code 337> (__DefaultInterrupt)
                  0x000044          0x4 LONG 0x1041c DEFINED (__Interrupt24)?<code 337> (__Interrupt24):<code 337> (__DefaultInterrupt)
                  0x000046          0x4 LONG 0x1041c DEFINED (__OC3Interrupt)?<code 337> (__OC3Interrupt):<code 337> (__DefaultInterrupt)
                  0x000048          0x4 LONG 0x1041c DEFINED (__OC4Interrupt)?<code 337> (__OC4Interrupt):<code 337> (__DefaultInterrupt)
                  0x00004a          0x4 LONG 0x1041c DEFINED (__T4Interrupt)?<code 337> (__T4Interrupt):<code 337> (__DefaultInterrupt)
                  0x00004c          0x4 LONG 0x1041c DEFINED (__T5Interrupt)?<code 337> (__T5Interrupt):<code 337> (__DefaultInterrupt)
                  0x00004e          0x4 LONG 0x1041c DEFINED (__INT2Interrupt)?<code 337> (__INT2Interrupt):<code 337> (__DefaultInterrupt)
                  0x000050          0x4 LONG 0xf49a DEFINED (__U2RXInterrupt)?<code 337> (__U2RXInterrupt):<code 337> (__DefaultInterrupt)
                  0x000052          0x4 LONG 0xf4d8 DEFINED (__U2TXInterrupt)?<code 337> (__U2TXInterrupt):<code 337> (__DefaultInterrupt)
                  0x000054          0x4 LONG 0x1041c DEFINED (__SPI2ErrInterrupt)?<code 337> (__SPI2ErrInterrupt):<code 337> (__DefaultInterrupt)
                  0x000056          0x4 LONG 0x1041c DEFINED (__SPI2Interrupt)?<code 337> (__SPI2Interrupt):<code 337> (__DefaultInterrupt)
                  0x000058          0x4 LONG 0x1041c DEFINED (__Interrupt34)?<code 337> (__Interrupt34):<code 337> (__DefaultInterrupt)
                  0x00005a          0x4 LONG 0x1041c DEFINED (__Interrupt35)?<code 337> (__Interrupt35):<code 337> (__DefaultInterrupt)
                  0x00005c          0x4 LONG 0x1041c DEFINED (__Interrupt36)?<code 337> (__Interrupt36):<code 337> (__DefaultInterrupt)
                  0x00005e          0x4 LONG 0x1041c DEFINED (__IC3Interrupt)?<code 337> (__IC3Interrupt):<code 337> (__DefaultInterrupt)
                  0x000060          0x4 LONG 0x1041c DEFINED (__IC4Interrupt)?<code 337> (__IC4Interrupt):<code 337> (__DefaultInterrupt)
                  0x000062          0x4 LONG 0x1041c DEFINED (__IC5Interrupt)?<code 337> (__IC5Interrupt):<code 337> (__DefaultInterrupt)
                  0x000064          0x4 LONG 0x1041c DEFINED (__Interrupt40)?<code 337> (__Interrupt40):<code 337> (__DefaultInterrupt)
                  0x000066          0x4 LONG 0x1041c DEFINED (__OC5Interrupt)?<code 337> (__OC5Interrupt):<code 337> (__DefaultInterrupt)
                  0x000068          0x4 LONG 0x1041c DEFINED (__Interrupt42)?<code 337> (__Interrupt42):<code 337> (__DefaultInterrupt)
                  0x00006a          0x4 LONG 0x1041c DEFINED (__Interrupt43)?<code 337> (__Interrupt43):<code 337> (__DefaultInterrupt)
                  0x00006c          0x4 LONG 0x1041c DEFINED (__Interrupt44)?<code 337> (__Interrupt44):<code 337> (__DefaultInterrupt)
                  0x00006e          0x4 LONG 0x1041c DEFINED (__PMPInterrupt)?<code 337> (__PMPInterrupt):<code 337> (__DefaultInterrupt)
                  0x000070          0x4 LONG 0x1041c DEFINED (__Interrupt46)?<code 337> (__Interrupt46):<code 337> (__DefaultInterrupt)
                  0x000072          0x4 LONG 0x1041c DEFINED (__Interrupt47)?<code 337> (__Interrupt47):<code 337> (__DefaultInterrupt)
                  0x000074          0x4 LONG 0x1041c DEFINED (__Interrupt48)?<code 337> (__Interrupt48):<code 337> (__DefaultInterrupt)
                  0x000076          0x4 LONG 0x1041c DEFINED (__SI2C2Interrupt)?<code 337> (__SI2C2Interrupt):<code 337> (__DefaultInterrupt)
                  0x000078          0x4 LONG 0x1041c DEFINED (__MI2C2Interrupt)?<code 337> (__MI2C2Interrupt):<code 337> (__DefaultInterrupt)
                  0x00007a          0x4 LONG 0x1041c DEFINED (__Interrupt51)?<code 337> (__Interrupt51):<code 337> (__DefaultInterrupt)
                  0x00007c          0x4 LONG 0x1041c DEFINED (__Interrupt52)?<code 337> (__Interrupt52):<code 337> (__DefaultInterrupt)
                  0x00007e          0x4 LONG 0x1041c DEFINED (__INT3Interrupt)?<code 337> (__INT3Interrupt):<code 337> (__DefaultInterrupt)
                  0x000080          0x4 LONG 0x1041c DEFINED (__INT4Interrupt)?<code 337> (__INT4Interrupt):<code 337> (__DefaultInterrupt)
                  0x000082          0x4 LONG 0x1041c DEFINED (__Interrupt55)?<code 337> (__Interrupt55):<code 337> (__DefaultInterrupt)
                  0x000084          0x4 LONG 0x1041c DEFINED (__Interrupt56)?<code 337> (__Interrupt56):<code 337> (__DefaultInterrupt)
                  0x000086          0x4 LONG 0x1041c DEFINED (__Interrupt57)?<code 337> (__Interrupt57):<code 337> (__DefaultInterrupt)
                  0x000088          0x4 LONG 0x1041c DEFINED (__Interrupt58)?<code 337> (__Interrupt58):<code 337> (__DefaultInterrupt)
                  0x00008a          0x4 LONG 0x1041c DEFINED (__Interrupt59)?<code 337> (__Interrupt59):<code 337> (__DefaultInterrupt)
                  0x00008c          0x4 LONG 0x1041c DEFINED (__Interrupt60)?<code 337> (__Interrupt60):<code 337> (__DefaultInterrupt)
                  0x00008e          0x4 LONG 0x1041c DEFINED (__Interrupt61)?<code 337> (__Interrupt61):<code 337> (__DefaultInterrupt)
                  0x000090          0x4 LONG 0x1041c DEFINED (__RTCCInterrupt)?<code 337> (__RTCCInterrupt):<code 337> (__DefaultInterrupt)
                  0x000092          0x4 LONG 0x1041c DEFINED (__Interrupt63)?<code 337> (__Interrupt63):<code 337> (__DefaultInterrupt)
                  0x000094          0x4 LONG 0x1041c DEFINED (__Interrupt64)?<code 337> (__Interrupt64):<code 337> (__DefaultInterrupt)
                  0x000096          0x4 LONG 0x1041c DEFINED (__U1ErrInterrupt)?<code 337> (__U1ErrInterrupt):<code 337> (__DefaultInterrupt)
                  0x000098          0x4 LONG 0x1041c DEFINED (__U2ErrInterrupt)?<code 337> (__U2ErrInterrupt):<code 337> (__DefaultInterrupt)
                  0x00009a          0x4 LONG 0x1041c DEFINED (__CRCInterrupt)?<code 337> (__CRCInterrupt):<code 337> (__DefaultInterrupt)
                  0x00009c          0x4 LONG 0x1041c DEFINED (__Interrupt68)?<code 337> (__Interrupt68):<code 337> (__DefaultInterrupt)
                  0x00009e          0x4 LONG 0x1041c DEFINED (__Interrupt69)?<code 337> (__Interrupt69):<code 337> (__DefaultInterrupt)
                  0x0000a0          0x4 LONG 0x1041c DEFINED (__Interrupt70)?<code 337> (__Interrupt70):<code 337> (__DefaultInterrupt)
                  0x0000a2          0x4 LONG 0x1041c DEFINED (__Interrupt71)?<code 337> (__Interrupt71):<code 337> (__DefaultInterrupt)
                  0x0000a4          0x4 LONG 0x1041c DEFINED (__Interrupt72)?<code 337> (__Interrupt72):<code 337> (__DefaultInterrupt)
                  0x0000a6          0x4 LONG 0x1041c DEFINED (__Interrupt73)?<code 337> (__Interrupt73):<code 337> (__DefaultInterrupt)
                  0x0000a8          0x4 LONG 0x1041c DEFINED (__Interrupt74)?<code 337> (__Interrupt74):<code 337> (__DefaultInterrupt)
                  0x0000aa          0x4 LONG 0x1041c DEFINED (__Interrupt75)?<code 337> (__Interrupt75):<code 337> (__DefaultInterrupt)
                  0x0000ac          0x4 LONG 0x1041c DEFINED (__Interrupt76)?<code 337> (__Interrupt76):<code 337> (__DefaultInterrupt)
                  0x0000ae          0x4 LONG 0x1041c DEFINED (__Interrupt77)?<code 337> (__Interrupt77):<code 337> (__DefaultInterrupt)
                  0x0000b0          0x4 LONG 0x1041c DEFINED (__Interrupt78)?<code 337> (__Interrupt78):<code 337> (__DefaultInterrupt)
                  0x0000b2          0x4 LONG 0x1041c DEFINED (__Interrupt79)?<code 337> (__Interrupt79):<code 337> (__DefaultInterrupt)
                  0x0000b4          0x4 LONG 0x1041c DEFINED (__Interrupt80)?<code 337> (__Interrupt80):<code 337> (__DefaultInterrupt)
                  0x0000b6          0x4 LONG 0x1041c DEFINED (__Interrupt81)?<code 337> (__Interrupt81):<code 337> (__DefaultInterrupt)
                  0x0000b8          0x4 LONG 0x1041c DEFINED (__Interrupt82)?<code 337> (__Interrupt82):<code 337> (__DefaultInterrupt)
                  0x0000ba          0x4 LONG 0x1041c DEFINED (__Interrupt83)?<code 337> (__Interrupt83):<code 337> (__DefaultInterrupt)
                  0x0000bc          0x4 LONG 0x1041c DEFINED (__Interrupt84)?<code 337> (__Interrupt84):<code 337> (__DefaultInterrupt)
                  0x0000be          0x4 LONG 0x1041c DEFINED (__Interrupt85)?<code 337> (__Interrupt85):<code 337> (__DefaultInterrupt)
                  0x0000c0          0x4 LONG 0x1041c DEFINED (__Interrupt86)?<code 337> (__Interrupt86):<code 337> (__DefaultInterrupt)
                  0x0000c2          0x4 LONG 0x1041c DEFINED (__Interrupt87)?<code 337> (__Interrupt87):<code 337> (__DefaultInterrupt)
                  0x0000c4          0x4 LONG 0x1041c DEFINED (__Interrupt88)?<code 337> (__Interrupt88):<code 337> (__DefaultInterrupt)
                  0x0000c6          0x4 LONG 0x1041c DEFINED (__Interrupt89)?<code 337> (__Interrupt89):<code 337> (__DefaultInterrupt)
                  0x0000c8          0x4 LONG 0x1041c DEFINED (__Interrupt90)?<code 337> (__Interrupt90):<code 337> (__DefaultInterrupt)
                  0x0000ca          0x4 LONG 0x1041c DEFINED (__Interrupt91)?<code 337> (__Interrupt91):<code 337> (__DefaultInterrupt)
                  0x0000cc          0x4 LONG 0x1041c DEFINED (__Interrupt92)?<code 337> (__Interrupt92):<code 337> (__DefaultInterrupt)
                  0x0000ce          0x4 LONG 0x1041c DEFINED (__Interrupt93)?<code 337> (__Interrupt93):<code 337> (__DefaultInterrupt)
                  0x0000d0          0x4 LONG 0x1041c DEFINED (__Interrupt94)?<code 337> (__Interrupt94):<code 337> (__DefaultInterrupt)
                  0x0000d2          0x4 LONG 0x1041c DEFINED (__Interrupt95)?<code 337> (__Interrupt95):<code 337> (__DefaultInterrupt)
                  0x0000d4          0x4 LONG 0x1041c DEFINED (__Interrupt96)?<code 337> (__Interrupt96):<code 337> (__DefaultInterrupt)
                  0x0000d6          0x4 LONG 0x1041c DEFINED (__Interrupt97)?<code 337> (__Interrupt97):<code 337> (__DefaultInterrupt)
                  0x0000d8          0x4 LONG 0x1041c DEFINED (__Interrupt98)?<code 337> (__Interrupt98):<code 337> (__DefaultInterrupt)
                  0x0000da          0x4 LONG 0x1041c DEFINED (__Interrupt99)?<code 337> (__Interrupt99):<code 337> (__DefaultInterrupt)
                  0x0000dc          0x4 LONG 0x1041c DEFINED (__Interrupt100)?<code 337> (__Interrupt100):<code 337> (__DefaultInterrupt)
                  0x0000de          0x4 LONG 0x1041c DEFINED (__Interrupt101)?<code 337> (__Interrupt101):<code 337> (__DefaultInterrupt)
                  0x0000e0          0x4 LONG 0x1041c DEFINED (__Interrupt102)?<code 337> (__Interrupt102):<code 337> (__DefaultInterrupt)
                  0x0000e2          0x4 LONG 0x1041c DEFINED (__Interrupt103)?<code 337> (__Interrupt103):<code 337> (__DefaultInterrupt)
                  0x0000e4          0x4 LONG 0x1041c DEFINED (__Interrupt104)?<code 337> (__Interrupt104):<code 337> (__DefaultInterrupt)
                  0x0000e6          0x4 LONG 0x1041c DEFINED (__Interrupt105)?<code 337> (__Interrupt105):<code 337> (__DefaultInterrupt)
                  0x0000e8          0x4 LONG 0x1041c DEFINED (__Interrupt106)?<code 337> (__Interrupt106):<code 337> (__DefaultInterrupt)
                  0x0000ea          0x4 LONG 0x1041c DEFINED (__Interrupt107)?<code 337> (__Interrupt107):<code 337> (__DefaultInterrupt)
                  0x0000ec          0x4 LONG 0x1041c DEFINED (__Interrupt108)?<code 337> (__Interrupt108):<code 337> (__DefaultInterrupt)
                  0x0000ee          0x4 LONG 0x1041c DEFINED (__Interrupt109)?<code 337> (__Interrupt109):<code 337> (__DefaultInterrupt)
                  0x0000f0          0x4 LONG 0x1041c DEFINED (__Interrupt110)?<code 337> (__Interrupt110):<code 337> (__DefaultInterrupt)
                  0x0000f2          0x4 LONG 0x1041c DEFINED (__Interrupt111)?<code 337> (__Interrupt111):<code 337> (__DefaultInterrupt)
                  0x0000f4          0x4 LONG 0x1041c DEFINED (__Interrupt112)?<code 337> (__Interrupt112):<code 337> (__DefaultInterrupt)
                  0x0000f6          0x4 LONG 0x1041c DEFINED (__Interrupt113)?<code 337> (__Interrupt113):<code 337> (__DefaultInterrupt)
                  0x0000f8          0x4 LONG 0x1041c DEFINED (__Interrupt114)?<code 337> (__Interrupt114):<code 337> (__DefaultInterrupt)
                  0x0000fa          0x4 LONG 0x1041c DEFINED (__Interrupt115)?<code 337> (__Interrupt115):<code 337> (__DefaultInterrupt)
                  0x0000fc          0x4 LONG 0x1041c DEFINED (__Interrupt116)?<code 337> (__Interrupt116):<code 337> (__DefaultInterrupt)
                  0x0000fe          0x4 LONG 0x1041c DEFINED (__Interrupt117)?<code 337> (__Interrupt117):<code 337> (__DefaultInterrupt)

.aivt             0x000104         0xfc
                  0x000104          0x4 LONG 0x1041c DEFINED (__AltReservedTrap0)?<code 337> (__AltReservedTrap0):DEFINED (__ReservedTrap0)?<code 337> (__ReservedTrap0):<code 337> (__DefaultInterrupt)
                  0x000106          0x4 LONG 0x1041c DEFINED (__AltOscillatorFail)?<code 337> (__AltOscillatorFail):DEFINED (__OscillatorFail)?<code 337> (__OscillatorFail):<code 337> (__DefaultInterrupt)
                  0x000108          0x4 LONG 0xcf8e DEFINED (__AltAddressError)?<code 337> (__AltAddressError):DEFINED (__AddressError)?<code 337> (__AddressError):<code 337> (__DefaultInterrupt)
                  0x00010a          0x4 LONG 0xcf98 DEFINED (__AltStackError)?<code 337> (__AltStackError):DEFINED (__StackError)?<code 337> (__StackError):<code 337> (__DefaultInterrupt)
                  0x00010c          0x4 LONG 0x1041c DEFINED (__AltMathError)?<code 337> (__AltMathError):DEFINED (__MathError)?<code 337> (__MathError):<code 337> (__DefaultInterrupt)
                  0x00010e          0x4 LONG 0x1041c DEFINED (__AltReservedTrap5)?<code 337> (__AltReservedTrap5):DEFINED (__ReservedTrap5)?<code 337> (__ReservedTrap5):<code 337> (__DefaultInterrupt)
                  0x000110          0x4 LONG 0x1041c DEFINED (__AltReservedTrap6)?<code 337> (__AltReservedTrap6):DEFINED (__ReservedTrap6)?<code 337> (__ReservedTrap6):<code 337> (__DefaultInterrupt)
                  0x000112          0x4 LONG 0x1041c DEFINED (__AltReservedTrap7)?<code 337> (__AltReservedTrap7):DEFINED (__ReservedTrap7)?<code 337> (__ReservedTrap7):<code 337> (__DefaultInterrupt)
                  0x000114          0x4 LONG 0x1041c DEFINED (__AltINT0Interrupt)?<code 337> (__AltINT0Interrupt):DEFINED (__INT0Interrupt)?<code 337> (__INT0Interrupt):<code 337> (__DefaultInterrupt)
                  0x000116          0x4 LONG 0x1041c DEFINED (__AltIC1Interrupt)?<code 337> (__AltIC1Interrupt):DEFINED (__IC1Interrupt)?<code 337> (__IC1Interrupt):<code 337> (__DefaultInterrupt)
                  0x000118          0x4 LONG 0x1041c DEFINED (__AltOC1Interrupt)?<code 337> (__AltOC1Interrupt):DEFINED (__OC1Interrupt)?<code 337> (__OC1Interrupt):<code 337> (__DefaultInterrupt)
                  0x00011a          0x4 LONG 0x10202 DEFINED (__AltT1Interrupt)?<code 337> (__AltT1Interrupt):DEFINED (__T1Interrupt)?<code 337> (__T1Interrupt):<code 337> (__DefaultInterrupt)
                  0x00011c          0x4 LONG 0x1041c DEFINED (__AltInterrupt4)?<code 337> (__AltInterrupt4):DEFINED (__Interrupt4)?<code 337> (__Interrupt4):<code 337> (__DefaultInterrupt)
                  0x00011e          0x4 LONG 0x1041c DEFINED (__AltIC2Interrupt)?<code 337> (__AltIC2Interrupt):DEFINED (__IC2Interrupt)?<code 337> (__IC2Interrupt):<code 337> (__DefaultInterrupt)
                  0x000120          0x4 LONG 0x1041c DEFINED (__AltOC2Interrupt)?<code 337> (__AltOC2Interrupt):DEFINED (__OC2Interrupt)?<code 337> (__OC2Interrupt):<code 337> (__DefaultInterrupt)
                  0x000122          0x4 LONG 0x1041c DEFINED (__AltT2Interrupt)?<code 337> (__AltT2Interrupt):DEFINED (__T2Interrupt)?<code 337> (__T2Interrupt):<code 337> (__DefaultInterrupt)
                  0x000124          0x4 LONG 0x1041c DEFINED (__AltT3Interrupt)?<code 337> (__AltT3Interrupt):DEFINED (__T3Interrupt)?<code 337> (__T3Interrupt):<code 337> (__DefaultInterrupt)
                  0x000126          0x4 LONG 0x1041c DEFINED (__AltSPI1ErrInterrupt)?<code 337> (__AltSPI1ErrInterrupt):DEFINED (__SPI1ErrInterrupt)?<code 337> (__SPI1ErrInterrupt):<code 337> (__DefaultInterrupt)
                  0x000128          0x4 LONG 0x1041c DEFINED (__AltSPI1Interrupt)?<code 337> (__AltSPI1Interrupt):DEFINED (__SPI1Interrupt)?<code 337> (__SPI1Interrupt):<code 337> (__DefaultInterrupt)
                  0x00012a          0x4 LONG 0x1041c DEFINED (__AltU1RXInterrupt)?<code 337> (__AltU1RXInterrupt):DEFINED (__U1RXInterrupt)?<code 337> (__U1RXInterrupt):<code 337> (__DefaultInterrupt)
                  0x00012c          0x4 LONG 0x1041c DEFINED (__AltU1TXInterrupt)?<code 337> (__AltU1TXInterrupt):DEFINED (__U1TXInterrupt)?<code 337> (__U1TXInterrupt):<code 337> (__DefaultInterrupt)
                  0x00012e          0x4 LONG 0x1041c DEFINED (__AltADC1Interrupt)?<code 337> (__AltADC1Interrupt):DEFINED (__ADC1Interrupt)?<code 337> (__ADC1Interrupt):<code 337> (__DefaultInterrupt)
                  0x000130          0x4 LONG 0x1041c DEFINED (__AltInterrupt14)?<code 337> (__AltInterrupt14):DEFINED (__Interrupt14)?<code 337> (__Interrupt14):<code 337> (__DefaultInterrupt)
                  0x000132          0x4 LONG 0x1041c DEFINED (__AltInterrupt15)?<code 337> (__AltInterrupt15):DEFINED (__Interrupt15)?<code 337> (__Interrupt15):<code 337> (__DefaultInterrupt)
                  0x000134          0x4 LONG 0x1041c DEFINED (__AltSI2C1Interrupt)?<code 337> (__AltSI2C1Interrupt):DEFINED (__SI2C1Interrupt)?<code 337> (__SI2C1Interrupt):<code 337> (__DefaultInterrupt)
                  0x000136          0x4 LONG 0x1041c DEFINED (__AltMI2C1Interrupt)?<code 337> (__AltMI2C1Interrupt):DEFINED (__MI2C1Interrupt)?<code 337> (__MI2C1Interrupt):<code 337> (__DefaultInterrupt)
                  0x000138          0x4 LONG 0x1041c DEFINED (__AltCompInterrupt)?<code 337> (__AltCompInterrupt):DEFINED (__CompInterrupt)?<code 337> (__CompInterrupt):<code 337> (__DefaultInterrupt)
                  0x00013a          0x4 LONG 0x1041c DEFINED (__AltCNInterrupt)?<code 337> (__AltCNInterrupt):DEFINED (__CNInterrupt)?<code 337> (__CNInterrupt):<code 337> (__DefaultInterrupt)
                  0x00013c          0x4 LONG 0x1041c DEFINED (__AltINT1Interrupt)?<code 337> (__AltINT1Interrupt):DEFINED (__INT1Interrupt)?<code 337> (__INT1Interrupt):<code 337> (__DefaultInterrupt)
                  0x00013e          0x4 LONG 0x1041c DEFINED (__AltInterrupt21)?<code 337> (__AltInterrupt21):DEFINED (__Interrupt21)?<code 337> (__Interrupt21):<code 337> (__DefaultInterrupt)
                  0x000140          0x4 LONG 0x1041c DEFINED (__AltInterrupt22)?<code 337> (__AltInterrupt22):DEFINED (__Interrupt22)?<code 337> (__Interrupt22):<code 337> (__DefaultInterrupt)
                  0x000142          0x4 LONG 0x1041c DEFINED (__AltInterrupt23)?<code 337> (__AltInterrupt23):DEFINED (__Interrupt23)?<code 337> (__Interrupt23):<code 337> (__DefaultInterrupt)
                  0x000144          0x4 LONG 0x1041c DEFINED (__AltInterrupt24)?<code 337> (__AltInterrupt24):DEFINED (__Interrupt24)?<code 337> (__Interrupt24):<code 337> (__DefaultInterrupt)
                  0x000146          0x4 LONG 0x1041c DEFINED (__AltOC3Interrupt)?<code 337> (__AltOC3Interrupt):DEFINED (__OC3Interrupt)?<code 337> (__OC3Interrupt):<code 337> (__DefaultInterrupt)
                  0x000148          0x4 LONG 0x1041c DEFINED (__AltOC4Interrupt)?<code 337> (__AltOC4Interrupt):DEFINED (__OC4Interrupt)?<code 337> (__OC4Interrupt):<code 337> (__DefaultInterrupt)
                  0x00014a          0x4 LONG 0x1041c DEFINED (__AltT4Interrupt)?<code 337> (__AltT4Interrupt):DEFINED (__T4Interrupt)?<code 337> (__T4Interrupt):<code 337> (__DefaultInterrupt)
                  0x00014c          0x4 LONG 0x1041c DEFINED (__AltT5Interrupt)?<code 337> (__AltT5Interrupt):DEFINED (__T5Interrupt)?<code 337> (__T5Interrupt):<code 337> (__DefaultInterrupt)
                  0x00014e          0x4 LONG 0x1041c DEFINED (__AltINT2Interrupt)?<code 337> (__AltINT2Interrupt):DEFINED (__INT2Interrupt)?<code 337> (__INT2Interrupt):<code 337> (__DefaultInterrupt)
                  0x000150          0x4 LONG 0xf49a DEFINED (__AltU2RXInterrupt)?<code 337> (__AltU2RXInterrupt):DEFINED (__U2RXInterrupt)?<code 337> (__U2RXInterrupt):<code 337> (__DefaultInterrupt)
                  0x000152          0x4 LONG 0xf4d8 DEFINED (__AltU2TXInterrupt)?<code 337> (__AltU2TXInterrupt):DEFINED (__U2TXInterrupt)?<code 337> (__U2TXInterrupt):<code 337> (__DefaultInterrupt)
                  0x000154          0x4 LONG 0x1041c DEFINED (__AltSPI2ErrInterrupt)?<code 337> (__AltSPI2ErrInterrupt):DEFINED (__SPI2ErrInterrupt)?<code 337> (__SPI2ErrInterrupt):<code 337> (__DefaultInterrupt)
                  0x000156          0x4 LONG 0x1041c DEFINED (__AltSPI2Interrupt)?<code 337> (__AltSPI2Interrupt):DEFINED (__SPI2Interrupt)?<code 337> (__SPI2Interrupt):<code 337> (__DefaultInterrupt)
                  0x000158          0x4 LONG 0x1041c DEFINED (__AltInterrupt34)?<code 337> (__AltInterrupt34):DEFINED (__Interrupt34)?<code 337> (__Interrupt34):<code 337> (__DefaultInterrupt)
                  0x00015a          0x4 LONG 0x1041c DEFINED (__AltInterrupt35)?<code 337> (__AltInterrupt35):DEFINED (__Interrupt35)?<code 337> (__Interrupt35):<code 337> (__DefaultInterrupt)
                  0x00015c          0x4 LONG 0x1041c DEFINED (__AltInterrupt36)?<code 337> (__AltInterrupt36):DEFINED (__Interrupt36)?<code 337> (__Interrupt36):<code 337> (__DefaultInterrupt)
                  0x00015e          0x4 LONG 0x1041c DEFINED (__AltIC3Interrupt)?<code 337> (__AltIC3Interrupt):DEFINED (__IC3Interrupt)?<code 337> (__IC3Interrupt):<code 337> (__DefaultInterrupt)
                  0x000160          0x4 LONG 0x1041c DEFINED (__AltIC4Interrupt)?<code 337> (__AltIC4Interrupt):DEFINED (__IC4Interrupt)?<code 337> (__IC4Interrupt):<code 337> (__DefaultInterrupt)
                  0x000162          0x4 LONG 0x1041c DEFINED (__AltIC5Interrupt)?<code 337> (__AltIC5Interrupt):DEFINED (__IC5Interrupt)?<code 337> (__IC5Interrupt):<code 337> (__DefaultInterrupt)
                  0x000164          0x4 LONG 0x1041c DEFINED (__AltInterrupt40)?<code 337> (__AltInterrupt40):DEFINED (__Interrupt40)?<code 337> (__Interrupt40):<code 337> (__DefaultInterrupt)
                  0x000166          0x4 LONG 0x1041c DEFINED (__AltOC5Interrupt)?<code 337> (__AltOC5Interrupt):DEFINED (__OC5Interrupt)?<code 337> (__OC5Interrupt):<code 337> (__DefaultInterrupt)
                  0x000168          0x4 LONG 0x1041c DEFINED (__AltInterrupt42)?<code 337> (__AltInterrupt42):DEFINED (__Interrupt42)?<code 337> (__Interrupt42):<code 337> (__DefaultInterrupt)
                  0x00016a          0x4 LONG 0x1041c DEFINED (__AltInterrupt43)?<code 337> (__AltInterrupt43):DEFINED (__Interrupt43)?<code 337> (__Interrupt43):<code 337> (__DefaultInterrupt)
                  0x00016c          0x4 LONG 0x1041c DEFINED (__AltInterrupt44)?<code 337> (__AltInterrupt44):DEFINED (__Interrupt44)?<code 337> (__Interrupt44):<code 337> (__DefaultInterrupt)
                  0x00016e          0x4 LONG 0x1041c DEFINED (__AltPMPInterrupt)?<code 337> (__AltPMPInterrupt):DEFINED (__PMPInterrupt)?<code 337> (__PMPInterrupt):<code 337> (__DefaultInterrupt)
                  0x000170          0x4 LONG 0x1041c DEFINED (__AltInterrupt46)?<code 337> (__AltInterrupt46):DEFINED (__Interrupt46)?<code 337> (__Interrupt46):<code 337> (__DefaultInterrupt)
                  0x000172          0x4 LONG 0x1041c DEFINED (__AltInterrupt47)?<code 337> (__AltInterrupt47):DEFINED (__Interrupt47)?<code 337> (__Interrupt47):<code 337> (__DefaultInterrupt)
                  0x000174          0x4 LONG 0x1041c DEFINED (__AltInterrupt48)?<code 337> (__AltInterrupt48):DEFINED (__Interrupt48)?<code 337> (__Interrupt48):<code 337> (__DefaultInterrupt)
                  0x000176          0x4 LONG 0x1041c DEFINED (__AltSI2C2Interrupt)?<code 337> (__AltSI2C2Interrupt):DEFINED (__SI2C2Interrupt)?<code 337> (__SI2C2Interrupt):<code 337> (__DefaultInterrupt)
                  0x000178          0x4 LONG 0x1041c DEFINED (__AltMI2C2Interrupt)?<code 337> (__AltMI2C2Interrupt):DEFINED (__MI2C2Interrupt)?<code 337> (__MI2C2Interrupt):<code 337> (__DefaultInterrupt)
                  0x00017a          0x4 LONG 0x1041c DEFINED (__AltInterrupt51)?<code 337> (__AltInterrupt51):DEFINED (__Interrupt51)?<code 337> (__Interrupt51):<code 337> (__DefaultInterrupt)
                  0x00017c          0x4 LONG 0x1041c DEFINED (__AltInterrupt52)?<code 337> (__AltInterrupt52):DEFINED (__Interrupt52)?<code 337> (__Interrupt52):<code 337> (__DefaultInterrupt)
                  0x00017e          0x4 LONG 0x1041c DEFINED (__AltINT3Interrupt)?<code 337> (__AltINT3Interrupt):DEFINED (__INT3Interrupt)?<code 337> (__INT3Interrupt):<code 337> (__DefaultInterrupt)
                  0x000180          0x4 LONG 0x1041c DEFINED (__AltINT4Interrupt)?<code 337> (__AltINT4Interrupt):DEFINED (__INT4Interrupt)?<code 337> (__INT4Interrupt):<code 337> (__DefaultInterrupt)
                  0x000182          0x4 LONG 0x1041c DEFINED (__AltInterrupt55)?<code 337> (__AltInterrupt55):DEFINED (__Interrupt55)?<code 337> (__Interrupt55):<code 337> (__DefaultInterrupt)
                  0x000184          0x4 LONG 0x1041c DEFINED (__AltInterrupt56)?<code 337> (__AltInterrupt56):DEFINED (__Interrupt56)?<code 337> (__Interrupt56):<code 337> (__DefaultInterrupt)
                  0x000186          0x4 LONG 0x1041c DEFINED (__AltInterrupt57)?<code 337> (__AltInterrupt57):DEFINED (__Interrupt57)?<code 337> (__Interrupt57):<code 337> (__DefaultInterrupt)
                  0x000188          0x4 LONG 0x1041c DEFINED (__AltInterrupt58)?<code 337> (__AltInterrupt58):DEFINED (__Interrupt58)?<code 337> (__Interrupt58):<code 337> (__DefaultInterrupt)
                  0x00018a          0x4 LONG 0x1041c DEFINED (__AltInterrupt59)?<code 337> (__AltInterrupt59):DEFINED (__Interrupt59)?<code 337> (__Interrupt59):<code 337> (__DefaultInterrupt)
                  0x00018c          0x4 LONG 0x1041c DEFINED (__AltInterrupt60)?<code 337> (__AltInterrupt60):DEFINED (__Interrupt60)?<code 337> (__Interrupt60):<code 337> (__DefaultInterrupt)
                  0x00018e          0x4 LONG 0x1041c DEFINED (__AltInterrupt61)?<code 337> (__AltInterrupt61):DEFINED (__Interrupt61)?<code 337> (__Interrupt61):<code 337> (__DefaultInterrupt)
                  0x000190          0x4 LONG 0x1041c DEFINED (__AltRTCCInterrupt)?<code 337> (__AltRTCCInterrupt):DEFINED (__RTCCInterrupt)?<code 337> (__RTCCInterrupt):<code 337> (__DefaultInterrupt)
                  0x000192          0x4 LONG 0x1041c DEFINED (__AltInterrupt63)?<code 337> (__AltInterrupt63):DEFINED (__Interrupt63)?<code 337> (__Interrupt63):<code 337> (__DefaultInterrupt)
                  0x000194          0x4 LONG 0x1041c DEFINED (__AltInterrupt64)?<code 337> (__AltInterrupt64):DEFINED (__Interrupt64)?<code 337> (__Interrupt64):<code 337> (__DefaultInterrupt)
                  0x000196          0x4 LONG 0x1041c DEFINED (__AltU1ErrInterrupt)?<code 337> (__AltU1ErrInterrupt):DEFINED (__U1ErrInterrupt)?<code 337> (__U1ErrInterrupt):<code 337> (__DefaultInterrupt)
                  0x000198          0x4 LONG 0x1041c DEFINED (__AltU2ErrInterrupt)?<code 337> (__AltU2ErrInterrupt):DEFINED (__U2ErrInterrupt)?<code 337> (__U2ErrInterrupt):<code 337> (__DefaultInterrupt)
                  0x00019a          0x4 LONG 0x1041c DEFINED (__AltCRCInterrupt)?<code 337> (__AltCRCInterrupt):DEFINED (__CRCInterrupt)?<code 337> (__CRCInterrupt):<code 337> (__DefaultInterrupt)
                  0x00019c          0x4 LONG 0x1041c DEFINED (__AltInterrupt68)?<code 337> (__AltInterrupt68):DEFINED (__Interrupt68)?<code 337> (__Interrupt68):<code 337> (__DefaultInterrupt)
                  0x00019e          0x4 LONG 0x1041c DEFINED (__AltInterrupt69)?<code 337> (__AltInterrupt69):DEFINED (__Interrupt69)?<code 337> (__Interrupt69):<code 337> (__DefaultInterrupt)
                  0x0001a0          0x4 LONG 0x1041c DEFINED (__AltInterrupt70)?<code 337> (__AltInterrupt70):DEFINED (__Interrupt70)?<code 337> (__Interrupt70):<code 337> (__DefaultInterrupt)
                  0x0001a2          0x4 LONG 0x1041c DEFINED (__AltInterrupt71)?<code 337> (__AltInterrupt71):DEFINED (__Interrupt71)?<code 337> (__Interrupt71):<code 337> (__DefaultInterrupt)
                  0x0001a4          0x4 LONG 0x1041c DEFINED (__AltInterrupt72)?<code 337> (__AltInterrupt72):DEFINED (__Interrupt72)?<code 337> (__Interrupt72):<code 337> (__DefaultInterrupt)
                  0x0001a6          0x4 LONG 0x1041c DEFINED (__AltInterrupt73)?<code 337> (__AltInterrupt73):DEFINED (__Interrupt73)?<code 337> (__Interrupt73):<code 337> (__DefaultInterrupt)
                  0x0001a8          0x4 LONG 0x1041c DEFINED (__AltInterrupt74)?<code 337> (__AltInterrupt74):DEFINED (__Interrupt74)?<code 337> (__Interrupt74):<code 337> (__DefaultInterrupt)
                  0x0001aa          0x4 LONG 0x1041c DEFINED (__AltInterrupt75)?<code 337> (__AltInterrupt75):DEFINED (__Interrupt75)?<code 337> (__Interrupt75):<code 337> (__DefaultInterrupt)
                  0x0001ac          0x4 LONG 0x1041c DEFINED (__AltInterrupt76)?<code 337> (__AltInterrupt76):DEFINED (__Interrupt76)?<code 337> (__Interrupt76):<code 337> (__DefaultInterrupt)
                  0x0001ae          0x4 LONG 0x1041c DEFINED (__AltInterrupt77)?<code 337> (__AltInterrupt77):DEFINED (__Interrupt77)?<code 337> (__Interrupt77):<code 337> (__DefaultInterrupt)
                  0x0001b0          0x4 LONG 0x1041c DEFINED (__AltInterrupt78)?<code 337> (__AltInterrupt78):DEFINED (__Interrupt78)?<code 337> (__Interrupt78):<code 337> (__DefaultInterrupt)
                  0x0001b2          0x4 LONG 0x1041c DEFINED (__AltInterrupt79)?<code 337> (__AltInterrupt79):DEFINED (__Interrupt79)?<code 337> (__Interrupt79):<code 337> (__DefaultInterrupt)
                  0x0001b4          0x4 LONG 0x1041c DEFINED (__AltInterrupt80)?<code 337> (__AltInterrupt80):DEFINED (__Interrupt80)?<code 337> (__Interrupt80):<code 337> (__DefaultInterrupt)
                  0x0001b6          0x4 LONG 0x1041c DEFINED (__AltInterrupt81)?<code 337> (__AltInterrupt81):DEFINED (__Interrupt81)?<code 337> (__Interrupt81):<code 337> (__DefaultInterrupt)
                  0x0001b8          0x4 LONG 0x1041c DEFINED (__AltInterrupt82)?<code 337> (__AltInterrupt82):DEFINED (__Interrupt82)?<code 337> (__Interrupt82):<code 337> (__DefaultInterrupt)
                  0x0001ba          0x4 LONG 0x1041c DEFINED (__AltInterrupt83)?<code 337> (__AltInterrupt83):DEFINED (__Interrupt83)?<code 337> (__Interrupt83):<code 337> (__DefaultInterrupt)
                  0x0001bc          0x4 LONG 0x1041c DEFINED (__AltInterrupt84)?<code 337> (__AltInterrupt84):DEFINED (__Interrupt84)?<code 337> (__Interrupt84):<code 337> (__DefaultInterrupt)
                  0x0001be          0x4 LONG 0x1041c DEFINED (__AltInterrupt85)?<code 337> (__AltInterrupt85):DEFINED (__Interrupt85)?<code 337> (__Interrupt85):<code 337> (__DefaultInterrupt)
                  0x0001c0          0x4 LONG 0x1041c DEFINED (__AltInterrupt86)?<code 337> (__AltInterrupt86):DEFINED (__Interrupt86)?<code 337> (__Interrupt86):<code 337> (__DefaultInterrupt)
                  0x0001c2          0x4 LONG 0x1041c DEFINED (__AltInterrupt87)?<code 337> (__AltInterrupt87):DEFINED (__Interrupt87)?<code 337> (__Interrupt87):<code 337> (__DefaultInterrupt)
                  0x0001c4          0x4 LONG 0x1041c DEFINED (__AltInterrupt88)?<code 337> (__AltInterrupt88):DEFINED (__Interrupt88)?<code 337> (__Interrupt88):<code 337> (__DefaultInterrupt)
                  0x0001c6          0x4 LONG 0x1041c DEFINED (__AltInterrupt89)?<code 337> (__AltInterrupt89):DEFINED (__Interrupt89)?<code 337> (__Interrupt89):<code 337> (__DefaultInterrupt)
                  0x0001c8          0x4 LONG 0x1041c DEFINED (__AltInterrupt90)?<code 337> (__AltInterrupt90):DEFINED (__Interrupt90)?<code 337> (__Interrupt90):<code 337> (__DefaultInterrupt)
                  0x0001ca          0x4 LONG 0x1041c DEFINED (__AltInterrupt91)?<code 337> (__AltInterrupt91):DEFINED (__Interrupt91)?<code 337> (__Interrupt91):<code 337> (__DefaultInterrupt)
                  0x0001cc          0x4 LONG 0x1041c DEFINED (__AltInterrupt92)?<code 337> (__AltInterrupt92):DEFINED (__Interrupt92)?<code 337> (__Interrupt92):<code 337> (__DefaultInterrupt)
                  0x0001ce          0x4 LONG 0x1041c DEFINED (__AltInterrupt93)?<code 337> (__AltInterrupt93):DEFINED (__Interrupt93)?<code 337> (__Interrupt93):<code 337> (__DefaultInterrupt)
                  0x0001d0          0x4 LONG 0x1041c DEFINED (__AltInterrupt94)?<code 337> (__AltInterrupt94):DEFINED (__Interrupt94)?<code 337> (__Interrupt94):<code 337> (__DefaultInterrupt)
                  0x0001d2          0x4 LONG 0x1041c DEFINED (__AltInterrupt95)?<code 337> (__AltInterrupt95):DEFINED (__Interrupt95)?<code 337> (__Interrupt95):<code 337> (__DefaultInterrupt)
                  0x0001d4          0x4 LONG 0x1041c DEFINED (__AltInterrupt96)?<code 337> (__AltInterrupt96):DEFINED (__Interrupt96)?<code 337> (__Interrupt96):<code 337> (__DefaultInterrupt)
                  0x0001d6          0x4 LONG 0x1041c DEFINED (__AltInterrupt97)?<code 337> (__AltInterrupt97):DEFINED (__Interrupt97)?<code 337> (__Interrupt97):<code 337> (__DefaultInterrupt)
                  0x0001d8          0x4 LONG 0x1041c DEFINED (__AltInterrupt98)?<code 337> (__AltInterrupt98):DEFINED (__Interrupt98)?<code 337> (__Interrupt98):<code 337> (__DefaultInterrupt)
                  0x0001da          0x4 LONG 0x1041c DEFINED (__AltInterrupt99)?<code 337> (__AltInterrupt99):DEFINED (__Interrupt99)?<code 337> (__Interrupt99):<code 337> (__DefaultInterrupt)
                  0x0001dc          0x4 LONG 0x1041c DEFINED (__AltInterrupt100)?<code 337> (__AltInterrupt100):DEFINED (__Interrupt100)?<code 337> (__Interrupt100):<code 337> (__DefaultInterrupt)
                  0x0001de          0x4 LONG 0x1041c DEFINED (__AltInterrupt101)?<code 337> (__AltInterrupt101):DEFINED (__Interrupt101)?<code 337> (__Interrupt101):<code 337> (__DefaultInterrupt)
                  0x0001e0          0x4 LONG 0x1041c DEFINED (__AltInterrupt102)?<code 337> (__AltInterrupt102):DEFINED (__Interrupt102)?<code 337> (__Interrupt102):<code 337> (__DefaultInterrupt)
                  0x0001e2          0x4 LONG 0x1041c DEFINED (__AltInterrupt103)?<code 337> (__AltInterrupt103):DEFINED (__Interrupt103)?<code 337> (__Interrupt103):<code 337> (__DefaultInterrupt)
                  0x0001e4          0x4 LONG 0x1041c DEFINED (__AltInterrupt104)?<code 337> (__AltInterrupt104):DEFINED (__Interrupt104)?<code 337> (__Interrupt104):<code 337> (__DefaultInterrupt)
                  0x0001e6          0x4 LONG 0x1041c DEFINED (__AltInterrupt105)?<code 337> (__AltInterrupt105):DEFINED (__Interrupt105)?<code 337> (__Interrupt105):<code 337> (__DefaultInterrupt)
                  0x0001e8          0x4 LONG 0x1041c DEFINED (__AltInterrupt106)?<code 337> (__AltInterrupt106):DEFINED (__Interrupt106)?<code 337> (__Interrupt106):<code 337> (__DefaultInterrupt)
                  0x0001ea          0x4 LONG 0x1041c DEFINED (__AltInterrupt107)?<code 337> (__AltInterrupt107):DEFINED (__Interrupt107)?<code 337> (__Interrupt107):<code 337> (__DefaultInterrupt)
                  0x0001ec          0x4 LONG 0x1041c DEFINED (__AltInterrupt108)?<code 337> (__AltInterrupt108):DEFINED (__Interrupt108)?<code 337> (__Interrupt108):<code 337> (__DefaultInterrupt)
                  0x0001ee          0x4 LONG 0x1041c DEFINED (__AltInterrupt109)?<code 337> (__AltInterrupt109):DEFINED (__Interrupt109)?<code 337> (__Interrupt109):<code 337> (__DefaultInterrupt)
                  0x0001f0          0x4 LONG 0x1041c DEFINED (__AltInterrupt110)?<code 337> (__AltInterrupt110):DEFINED (__Interrupt110)?<code 337> (__Interrupt110):<code 337> (__DefaultInterrupt)
                  0x0001f2          0x4 LONG 0x1041c DEFINED (__AltInterrupt111)?<code 337> (__AltInterrupt111):DEFINED (__Interrupt111)?<code 337> (__Interrupt111):<code 337> (__DefaultInterrupt)
                  0x0001f4          0x4 LONG 0x1041c DEFINED (__AltInterrupt112)?<code 337> (__AltInterrupt112):DEFINED (__Interrupt112)?<code 337> (__Interrupt112):<code 337> (__DefaultInterrupt)
                  0x0001f6          0x4 LONG 0x1041c DEFINED (__AltInterrupt113)?<code 337> (__AltInterrupt113):DEFINED (__Interrupt113)?<code 337> (__Interrupt113):<code 337> (__DefaultInterrupt)
                  0x0001f8          0x4 LONG 0x1041c DEFINED (__AltInterrupt114)?<code 337> (__AltInterrupt114):DEFINED (__Interrupt114)?<code 337> (__Interrupt114):<code 337> (__DefaultInterrupt)
                  0x0001fa          0x4 LONG 0x1041c DEFINED (__AltInterrupt115)?<code 337> (__AltInterrupt115):DEFINED (__Interrupt115)?<code 337> (__Interrupt115):<code 337> (__DefaultInterrupt)
                  0x0001fc          0x4 LONG 0x1041c DEFINED (__AltInterrupt116)?<code 337> (__AltInterrupt116):DEFINED (__Interrupt116)?<code 337> (__Interrupt116):<code 337> (__DefaultInterrupt)
                  0x0001fe          0x4 LONG 0x1041c DEFINED (__AltInterrupt117)?<code 337> (__AltInterrupt117):DEFINED (__Interrupt117)?<code 337> (__Interrupt117):<code 337> (__DefaultInterrupt)
                    0x0000                  WREG0 = 0x0
                    0x0000                  _WREG0 = 0x0
                    0x0002                  WREG1 = 0x2
                    0x0002                  _WREG1 = 0x2
                    0x0004                  WREG2 = 0x4
                    0x0004                  _WREG2 = 0x4
                    0x0006                  WREG3 = 0x6
                    0x0006                  _WREG3 = 0x6
                    0x0008                  WREG4 = 0x8
                    0x0008                  _WREG4 = 0x8
                    0x000a                  WREG5 = 0xa
                    0x000a                  _WREG5 = 0xa
                    0x000c                  WREG6 = 0xc
                    0x000c                  _WREG6 = 0xc
                    0x000e                  WREG7 = 0xe
                    0x000e                  _WREG7 = 0xe
                    0x0010                  WREG8 = 0x10
                    0x0010                  _WREG8 = 0x10
                    0x0012                  WREG9 = 0x12
                    0x0012                  _WREG9 = 0x12
                    0x0014                  WREG10 = 0x14
                    0x0014                  _WREG10 = 0x14
                    0x0016                  WREG11 = 0x16
                    0x0016                  _WREG11 = 0x16
                    0x0018                  WREG12 = 0x18
                    0x0018                  _WREG12 = 0x18
                    0x001a                  WREG13 = 0x1a
                    0x001a                  _WREG13 = 0x1a
                    0x001c                  WREG14 = 0x1c
                    0x001c                  _WREG14 = 0x1c
                    0x001e                  WREG15 = 0x1e
                    0x001e                  _WREG15 = 0x1e
                    0x0020                  SPLIM = 0x20
                    0x0020                  _SPLIM = 0x20
                    0x002e                  PCL = 0x2e
                    0x002e                  _PCL = 0x2e
                    0x0030                  PCH = 0x30
                    0x0030                  _PCH = 0x30
                    0x0032                  TBLPAG = 0x32
                    0x0032                  _TBLPAG = 0x32
                    0x0034                  PSVPAG = 0x34
                    0x0034                  _PSVPAG = 0x34
                    0x0036                  RCOUNT = 0x36
                    0x0036                  _RCOUNT = 0x36
                    0x0042                  SR = 0x42
                    0x0042                  _SR = 0x42
                    0x0042                  _SRbits = 0x42
                    0x0044                  CORCON = 0x44
                    0x0044                  _CORCON = 0x44
                    0x0044                  _CORCONbits = 0x44
                    0x0052                  DISICNT = 0x52
                    0x0052                  _DISICNT = 0x52
                    0x0060                  CNEN1 = 0x60
                    0x0060                  _CNEN1 = 0x60
                    0x0060                  _CNEN1bits = 0x60
                    0x0062                  CNEN2 = 0x62
                    0x0062                  _CNEN2 = 0x62
                    0x0062                  _CNEN2bits = 0x62
                    0x0068                  CNPU1 = 0x68
                    0x0068                  _CNPU1 = 0x68
                    0x0068                  _CNPU1bits = 0x68
                    0x006a                  CNPU2 = 0x6a
                    0x006a                  _CNPU2 = 0x6a
                    0x006a                  _CNPU2bits = 0x6a
                    0x0080                  INTCON1 = 0x80
                    0x0080                  _INTCON1 = 0x80
                    0x0080                  _INTCON1bits = 0x80
                    0x0082                  INTCON2 = 0x82
                    0x0082                  _INTCON2 = 0x82
                    0x0082                  _INTCON2bits = 0x82
                    0x0084                  IFS0 = 0x84
                    0x0084                  _IFS0 = 0x84
                    0x0084                  _IFS0bits = 0x84
                    0x0086                  IFS1 = 0x86
                    0x0086                  _IFS1 = 0x86
                    0x0086                  _IFS1bits = 0x86
                    0x0088                  IFS2 = 0x88
                    0x0088                  _IFS2 = 0x88
                    0x0088                  _IFS2bits = 0x88
                    0x008a                  IFS3 = 0x8a
                    0x008a                  _IFS3 = 0x8a
                    0x008a                  _IFS3bits = 0x8a
                    0x008c                  IFS4 = 0x8c
                    0x008c                  _IFS4 = 0x8c
                    0x008c                  _IFS4bits = 0x8c
                    0x0094                  IEC0 = 0x94
                    0x0094                  _IEC0 = 0x94
                    0x0094                  _IEC0bits = 0x94
                    0x0096                  IEC1 = 0x96
                    0x0096                  _IEC1 = 0x96
                    0x0096                  _IEC1bits = 0x96
                    0x0098                  IEC2 = 0x98
                    0x0098                  _IEC2 = 0x98
                    0x0098                  _IEC2bits = 0x98
                    0x009a                  IEC3 = 0x9a
                    0x009a                  _IEC3 = 0x9a
                    0x009a                  _IEC3bits = 0x9a
                    0x009c                  IEC4 = 0x9c
                    0x009c                  _IEC4 = 0x9c
                    0x009c                  _IEC4bits = 0x9c
                    0x00a4                  IPC0 = 0xa4
                    0x00a4                  _IPC0 = 0xa4
                    0x00a4                  _IPC0bits = 0xa4
                    0x00a6                  IPC1 = 0xa6
                    0x00a6                  _IPC1 = 0xa6
                    0x00a6                  _IPC1bits = 0xa6
                    0x00a8                  IPC2 = 0xa8
                    0x00a8                  _IPC2 = 0xa8
                    0x00a8                  _IPC2bits = 0xa8
                    0x00aa                  IPC3 = 0xaa
                    0x00aa                  _IPC3 = 0xaa
                    0x00aa                  _IPC3bits = 0xaa
                    0x00ac                  IPC4 = 0xac
                    0x00ac                  _IPC4 = 0xac
                    0x00ac                  _IPC4bits = 0xac
                    0x00ae                  IPC5 = 0xae
                    0x00ae                  _IPC5 = 0xae
                    0x00ae                  _IPC5bits = 0xae
                    0x00b0                  IPC6 = 0xb0
                    0x00b0                  _IPC6 = 0xb0
                    0x00b0                  _IPC6bits = 0xb0
                    0x00b2                  IPC7 = 0xb2
                    0x00b2                  _IPC7 = 0xb2
                    0x00b2                  _IPC7bits = 0xb2
                    0x00b4                  IPC8 = 0xb4
                    0x00b4                  _IPC8 = 0xb4
                    0x00b4                  _IPC8bits = 0xb4
                    0x00b6                  IPC9 = 0xb6
                    0x00b6                  _IPC9 = 0xb6
                    0x00b6                  _IPC9bits = 0xb6
                    0x00b8                  IPC10 = 0xb8
                    0x00b8                  _IPC10 = 0xb8
                    0x00b8                  _IPC10bits = 0xb8
                    0x00ba                  IPC11 = 0xba
                    0x00ba                  _IPC11 = 0xba
                    0x00ba                  _IPC11bits = 0xba
                    0x00bc                  IPC12 = 0xbc
                    0x00bc                  _IPC12 = 0xbc
                    0x00bc                  _IPC12bits = 0xbc
                    0x00be                  IPC13 = 0xbe
                    0x00be                  _IPC13 = 0xbe
                    0x00be                  _IPC13bits = 0xbe
                    0x00c2                  IPC15 = 0xc2
                    0x00c2                  _IPC15 = 0xc2
                    0x00c2                  _IPC15bits = 0xc2
                    0x00c4                  IPC16 = 0xc4
                    0x00c4                  _IPC16 = 0xc4
                    0x00c4                  _IPC16bits = 0xc4
                    0x0100                  TMR1 = 0x100
                    0x0100                  _TMR1 = 0x100
                    0x0102                  PR1 = 0x102
                    0x0102                  _PR1 = 0x102
                    0x0104                  T1CON = 0x104
                    0x0104                  _T1CON = 0x104
                    0x0104                  _T1CONbits = 0x104
                    0x0106                  TMR2 = 0x106
                    0x0106                  _TMR2 = 0x106
                    0x0108                  TMR3HLD = 0x108
                    0x0108                  _TMR3HLD = 0x108
                    0x010a                  TMR3 = 0x10a
                    0x010a                  _TMR3 = 0x10a
                    0x010c                  PR2 = 0x10c
                    0x010c                  _PR2 = 0x10c
                    0x010e                  PR3 = 0x10e
                    0x010e                  _PR3 = 0x10e
                    0x0110                  T2CON = 0x110
                    0x0110                  _T2CON = 0x110
                    0x0110                  _T2CONbits = 0x110
                    0x0112                  T3CON = 0x112
                    0x0112                  _T3CON = 0x112
                    0x0112                  _T3CONbits = 0x112
                    0x0114                  TMR4 = 0x114
                    0x0114                  _TMR4 = 0x114
                    0x0116                  TMR5HLD = 0x116
                    0x0116                  _TMR5HLD = 0x116
                    0x0118                  TMR5 = 0x118
                    0x0118                  _TMR5 = 0x118
                    0x011a                  PR4 = 0x11a
                    0x011a                  _PR4 = 0x11a
                    0x011c                  PR5 = 0x11c
                    0x011c                  _PR5 = 0x11c
                    0x011e                  T4CON = 0x11e
                    0x011e                  _T4CON = 0x11e
                    0x011e                  _T4CONbits = 0x11e
                    0x0120                  T5CON = 0x120
                    0x0120                  _T5CON = 0x120
                    0x0120                  _T5CONbits = 0x120
                    0x0140                  IC1BUF = 0x140
                    0x0140                  _IC1BUF = 0x140
                    0x0142                  IC1CON = 0x142
                    0x0142                  _IC1CON = 0x142
                    0x0142                  _IC1CONbits = 0x142
                    0x0144                  IC2BUF = 0x144
                    0x0144                  _IC2BUF = 0x144
                    0x0146                  IC2CON = 0x146
                    0x0146                  _IC2CON = 0x146
                    0x0146                  _IC2CONbits = 0x146
                    0x0148                  IC3BUF = 0x148
                    0x0148                  _IC3BUF = 0x148
                    0x014a                  IC3CON = 0x14a
                    0x014a                  _IC3CON = 0x14a
                    0x014a                  _IC3CONbits = 0x14a
                    0x014c                  IC4BUF = 0x14c
                    0x014c                  _IC4BUF = 0x14c
                    0x014e                  IC4CON = 0x14e
                    0x014e                  _IC4CON = 0x14e
                    0x014e                  _IC4CONbits = 0x14e
                    0x0150                  IC5BUF = 0x150
                    0x0150                  _IC5BUF = 0x150
                    0x0152                  IC5CON = 0x152
                    0x0152                  _IC5CON = 0x152
                    0x0152                  _IC5CONbits = 0x152
                    0x0180                  OC1RS = 0x180
                    0x0180                  _OC1RS = 0x180
                    0x0182                  OC1R = 0x182
                    0x0182                  _OC1R = 0x182
                    0x0184                  OC1CON = 0x184
                    0x0184                  _OC1CON = 0x184
                    0x0184                  _OC1CONbits = 0x184
                    0x0186                  OC2RS = 0x186
                    0x0186                  _OC2RS = 0x186
                    0x0188                  OC2R = 0x188
                    0x0188                  _OC2R = 0x188
                    0x018a                  OC2CON = 0x18a
                    0x018a                  _OC2CON = 0x18a
                    0x018a                  _OC2CONbits = 0x18a
                    0x018c                  OC3RS = 0x18c
                    0x018c                  _OC3RS = 0x18c
                    0x018e                  OC3R = 0x18e
                    0x018e                  _OC3R = 0x18e
                    0x0190                  OC3CON = 0x190
                    0x0190                  _OC3CON = 0x190
                    0x0190                  _OC3CONbits = 0x190
                    0x0192                  OC4RS = 0x192
                    0x0192                  _OC4RS = 0x192
                    0x0194                  OC4R = 0x194
                    0x0194                  _OC4R = 0x194
                    0x0196                  OC4CON = 0x196
                    0x0196                  _OC4CON = 0x196
                    0x0196                  _OC4CONbits = 0x196
                    0x0198                  OC5RS = 0x198
                    0x0198                  _OC5RS = 0x198
                    0x019a                  OC5R = 0x19a
                    0x019a                  _OC5R = 0x19a
                    0x019c                  OC5CON = 0x19c
                    0x019c                  _OC5CON = 0x19c
                    0x019c                  _OC5CONbits = 0x19c
                    0x0200                  I2C1RCV = 0x200
                    0x0200                  _I2C1RCV = 0x200
                    0x0202                  I2C1TRN = 0x202
                    0x0202                  _I2C1TRN = 0x202
                    0x0204                  I2C1BRG = 0x204
                    0x0204                  _I2C1BRG = 0x204
                    0x0206                  I2C1CON = 0x206
                    0x0206                  _I2C1CON = 0x206
                    0x0206                  _I2C1CONbits = 0x206
                    0x0208                  I2C1STAT = 0x208
                    0x0208                  _I2C1STAT = 0x208
                    0x0208                  _I2C1STATbits = 0x208
                    0x020a                  I2C1ADD = 0x20a
                    0x020a                  _I2C1ADD = 0x20a
                    0x020c                  I2C1MSK = 0x20c
                    0x020c                  _I2C1MSK = 0x20c
                    0x0210                  I2C2RCV = 0x210
                    0x0210                  _I2C2RCV = 0x210
                    0x0212                  I2C2TRN = 0x212
                    0x0212                  _I2C2TRN = 0x212
                    0x0214                  I2C2BRG = 0x214
                    0x0214                  _I2C2BRG = 0x214
                    0x0216                  I2C2CON = 0x216
                    0x0216                  _I2C2CON = 0x216
                    0x0216                  _I2C2CONbits = 0x216
                    0x0218                  I2C2STAT = 0x218
                    0x0218                  _I2C2STAT = 0x218
                    0x0218                  _I2C2STATbits = 0x218
                    0x021a                  I2C2ADD = 0x21a
                    0x021a                  _I2C2ADD = 0x21a
                    0x021c                  I2C2MSK = 0x21c
                    0x021c                  _I2C2MSK = 0x21c
                    0x0220                  U1MODE = 0x220
                    0x0220                  _U1MODE = 0x220
                    0x0220                  _U1MODEbits = 0x220
                    0x0222                  U1STA = 0x222
                    0x0222                  _U1STA = 0x222
                    0x0222                  _U1STAbits = 0x222
                    0x0224                  U1TXREG = 0x224
                    0x0224                  _U1TXREG = 0x224
                    0x0226                  U1RXREG = 0x226
                    0x0226                  _U1RXREG = 0x226
                    0x0228                  U1BRG = 0x228
                    0x0228                  _U1BRG = 0x228
                    0x0230                  U2MODE = 0x230
                    0x0230                  _U2MODE = 0x230
                    0x0230                  _U2MODEbits = 0x230
                    0x0232                  U2STA = 0x232
                    0x0232                  _U2STA = 0x232
                    0x0232                  _U2STAbits = 0x232
                    0x0234                  U2TXREG = 0x234
                    0x0234                  _U2TXREG = 0x234
                    0x0236                  U2RXREG = 0x236
                    0x0236                  _U2RXREG = 0x236
                    0x0238                  U2BRG = 0x238
                    0x0238                  _U2BRG = 0x238
                    0x0240                  SPI1STAT = 0x240
                    0x0240                  _SPI1STAT = 0x240
                    0x0240                  _SPI1STATbits = 0x240
                    0x0242                  SPI1CON1 = 0x242
                    0x0242                  _SPI1CON1 = 0x242
                    0x0242                  _SPI1CON1bits = 0x242
                    0x0244                  SPI1CON2 = 0x244
                    0x0244                  _SPI1CON2 = 0x244
                    0x0244                  _SPI1CON2bits = 0x244
                    0x0248                  SPI1BUF = 0x248
                    0x0248                  _SPI1BUF = 0x248
                    0x0260                  SPI2STAT = 0x260
                    0x0260                  _SPI2STAT = 0x260
                    0x0260                  _SPI2STATbits = 0x260
                    0x0262                  SPI2CON1 = 0x262
                    0x0262                  _SPI2CON1 = 0x262
                    0x0262                  _SPI2CON1bits = 0x262
                    0x0264                  SPI2CON2 = 0x264
                    0x0264                  _SPI2CON2 = 0x264
                    0x0264                  _SPI2CON2bits = 0x264
                    0x0268                  SPI2BUF = 0x268
                    0x0268                  _SPI2BUF = 0x268
                    0x02c0                  TRISA = 0x2c0
                    0x02c0                  _TRISA = 0x2c0
                    0x02c0                  _TRISAbits = 0x2c0
                    0x02c2                  PORTA = 0x2c2
                    0x02c2                  _PORTA = 0x2c2
                    0x02c2                  _PORTAbits = 0x2c2
                    0x02c4                  LATA = 0x2c4
                    0x02c4                  _LATA = 0x2c4
                    0x02c4                  _LATAbits = 0x2c4
                    0x02c6                  TRISB = 0x2c6
                    0x02c6                  _TRISB = 0x2c6
                    0x02c6                  _TRISBbits = 0x2c6
                    0x02c8                  PORTB = 0x2c8
                    0x02c8                  _PORTB = 0x2c8
                    0x02c8                  _PORTBbits = 0x2c8
                    0x02ca                  LATB = 0x2ca
                    0x02ca                  _LATB = 0x2ca
                    0x02ca                  _LATBbits = 0x2ca
                    0x02cc                  TRISC = 0x2cc
                    0x02cc                  _TRISC = 0x2cc
                    0x02cc                  _TRISCbits = 0x2cc
                    0x02ce                  PORTC = 0x2ce
                    0x02ce                  _PORTC = 0x2ce
                    0x02ce                  _PORTCbits = 0x2ce
                    0x02d0                  LATC = 0x2d0
                    0x02d0                  _LATC = 0x2d0
                    0x02d0                  _LATCbits = 0x2d0
                    0x02d2                  TRISD = 0x2d2
                    0x02d2                  _TRISD = 0x2d2
                    0x02d2                  _TRISDbits = 0x2d2
                    0x02d4                  PORTD = 0x2d4
                    0x02d4                  _PORTD = 0x2d4
                    0x02d4                  _PORTDbits = 0x2d4
                    0x02d6                  LATD = 0x2d6
                    0x02d6                  _LATD = 0x2d6
                    0x02d6                  _LATDbits = 0x2d6
                    0x02d8                  TRISE = 0x2d8
                    0x02d8                  _TRISE = 0x2d8
                    0x02d8                  _TRISEbits = 0x2d8
                    0x02da                  PORTE = 0x2da
                    0x02da                  _PORTE = 0x2da
                    0x02da                  _PORTEbits = 0x2da
                    0x02dc                  LATE = 0x2dc
                    0x02dc                  _LATE = 0x2dc
                    0x02dc                  _LATEbits = 0x2dc
                    0x02de                  TRISF = 0x2de
                    0x02de                  _TRISF = 0x2de
                    0x02de                  _TRISFbits = 0x2de
                    0x02e0                  PORTF = 0x2e0
                    0x02e0                  _PORTF = 0x2e0
                    0x02e0                  _PORTFbits = 0x2e0
                    0x02e2                  LATF = 0x2e2
                    0x02e2                  _LATF = 0x2e2
                    0x02e2                  _LATFbits = 0x2e2
                    0x02e4                  TRISG = 0x2e4
                    0x02e4                  _TRISG = 0x2e4
                    0x02e4                  _TRISGbits = 0x2e4
                    0x02e6                  PORTG = 0x2e6
                    0x02e6                  _PORTG = 0x2e6
                    0x02e6                  _PORTGbits = 0x2e6
                    0x02e8                  LATG = 0x2e8
                    0x02e8                  _LATG = 0x2e8
                    0x02e8                  _LATGbits = 0x2e8
                    0x02fc                  PADCFG1 = 0x2fc
                    0x02fc                  _PADCFG1 = 0x2fc
                    0x02fc                  _PADCFG1bits = 0x2fc
                    0x0300                  ADC1BUF0 = 0x300
                    0x0300                  _ADC1BUF0 = 0x300
                    0x0302                  ADC1BUF1 = 0x302
                    0x0302                  _ADC1BUF1 = 0x302
                    0x0304                  ADC1BUF2 = 0x304
                    0x0304                  _ADC1BUF2 = 0x304
                    0x0306                  ADC1BUF3 = 0x306
                    0x0306                  _ADC1BUF3 = 0x306
                    0x0308                  ADC1BUF4 = 0x308
                    0x0308                  _ADC1BUF4 = 0x308
                    0x030a                  ADC1BUF5 = 0x30a
                    0x030a                  _ADC1BUF5 = 0x30a
                    0x030c                  ADC1BUF6 = 0x30c
                    0x030c                  _ADC1BUF6 = 0x30c
                    0x030e                  ADC1BUF7 = 0x30e
                    0x030e                  _ADC1BUF7 = 0x30e
                    0x0310                  ADC1BUF8 = 0x310
                    0x0310                  _ADC1BUF8 = 0x310
                    0x0312                  ADC1BUF9 = 0x312
                    0x0312                  _ADC1BUF9 = 0x312
                    0x0314                  ADC1BUFA = 0x314
                    0x0314                  _ADC1BUFA = 0x314
                    0x0316                  ADC1BUFB = 0x316
                    0x0316                  _ADC1BUFB = 0x316
                    0x0318                  ADC1BUFC = 0x318
                    0x0318                  _ADC1BUFC = 0x318
                    0x031a                  ADC1BUFD = 0x31a
                    0x031a                  _ADC1BUFD = 0x31a
                    0x031c                  ADC1BUFE = 0x31c
                    0x031c                  _ADC1BUFE = 0x31c
                    0x031e                  ADC1BUFF = 0x31e
                    0x031e                  _ADC1BUFF = 0x31e
                    0x0320                  AD1CON1 = 0x320
                    0x0320                  _AD1CON1 = 0x320
                    0x0320                  _AD1CON1bits = 0x320
                    0x0322                  AD1CON2 = 0x322
                    0x0322                  _AD1CON2 = 0x322
                    0x0322                  _AD1CON2bits = 0x322
                    0x0324                  AD1CON3 = 0x324
                    0x0324                  _AD1CON3 = 0x324
                    0x0324                  _AD1CON3bits = 0x324
                    0x0328                  AD1CHS = 0x328
                    0x0328                  _AD1CHS = 0x328
                    0x0328                  _AD1CHSbits = 0x328
                    0x032c                  AD1PCFG = 0x32c
                    0x032c                  _AD1PCFG = 0x32c
                    0x032c                  _AD1PCFGbits = 0x32c
                    0x0330                  AD1CSSL = 0x330
                    0x0330                  _AD1CSSL = 0x330
                    0x0330                  _AD1CSSLbits = 0x330
                    0x0600                  PMCON = 0x600
                    0x0600                  _PMCON = 0x600
                    0x0600                  _PMCONbits = 0x600
                    0x0602                  PMMODE = 0x602
                    0x0602                  _PMMODE = 0x602
                    0x0602                  _PMMODEbits = 0x602
                    0x0604                  PMADDR = 0x604
                    0x0604                  _PMADDR = 0x604
                    0x0604                  _PMADDRbits = 0x604
                    0x0604                  PMDOUT1 = 0x604
                    0x0604                  _PMDOUT1 = 0x604
                    0x0604                  _PMDOUT1bits = 0x604
                    0x0606                  PMDOUT2 = 0x606
                    0x0606                  _PMDOUT2 = 0x606
                    0x0608                  PMDIN1 = 0x608
                    0x0608                  _PMDIN1 = 0x608
                    0x060a                  PMDIN2 = 0x60a
                    0x060a                  _PMDIN2 = 0x60a
                    0x060c                  PMAEN = 0x60c
                    0x060c                  _PMAEN = 0x60c
                    0x060c                  _PMAENbits = 0x60c
                    0x060e                  PMSTAT = 0x60e
                    0x060e                  _PMSTAT = 0x60e
                    0x060e                  _PMSTATbits = 0x60e
                    0x0620                  ALRMVAL = 0x620
                    0x0620                  _ALRMVAL = 0x620
                    0x0622                  ALCFGRPT = 0x622
                    0x0622                  _ALCFGRPT = 0x622
                    0x0622                  _ALCFGRPTbits = 0x622
                    0x0624                  RTCVAL = 0x624
                    0x0624                  _RTCVAL = 0x624
                    0x0626                  RCFGCAL = 0x626
                    0x0626                  _RCFGCAL = 0x626
                    0x0626                  _RCFGCALbits = 0x626
                    0x0630                  CMCON = 0x630
                    0x0630                  _CMCON = 0x630
                    0x0630                  _CMCONbits = 0x630
                    0x0632                  CVRCON = 0x632
                    0x0632                  _CVRCON = 0x632
                    0x0632                  _CVRCONbits = 0x632
                    0x0640                  CRCCON = 0x640
                    0x0640                  _CRCCON = 0x640
                    0x0640                  _CRCCONbits = 0x640
                    0x0642                  CRCXOR = 0x642
                    0x0642                  _CRCXOR = 0x642
                    0x0642                  _CRCXORbits = 0x642
                    0x0644                  CRCDAT = 0x644
                    0x0644                  _CRCDAT = 0x644
                    0x0646                  CRCWDAT = 0x646
                    0x0646                  _CRCWDAT = 0x646
                    0x06c0                  ODCA = 0x6c0
                    0x06c0                  _ODCA = 0x6c0
                    0x06c0                  _ODCAbits = 0x6c0
                    0x06c6                  ODCB = 0x6c6
                    0x06c6                  _ODCB = 0x6c6
                    0x06c6                  _ODCBbits = 0x6c6
                    0x06cc                  ODCC = 0x6cc
                    0x06cc                  _ODCC = 0x6cc
                    0x06cc                  _ODCCbits = 0x6cc
                    0x06d2                  ODCD = 0x6d2
                    0x06d2                  _ODCD = 0x6d2
                    0x06d2                  _ODCDbits = 0x6d2
                    0x06d8                  ODCE = 0x6d8
                    0x06d8                  _ODCE = 0x6d8
                    0x06d8                  _ODCEbits = 0x6d8
                    0x06de                  ODCF = 0x6de
                    0x06de                  _ODCF = 0x6de
                    0x06de                  _ODCFbits = 0x6de
                    0x06e4                  ODCG = 0x6e4
                    0x06e4                  _ODCG = 0x6e4
                    0x06e4                  _ODCGbits = 0x6e4
                    0x0740                  RCON = 0x740
                    0x0740                  _RCON = 0x740
                    0x0740                  _RCONbits = 0x740
                    0x0742                  OSCCON = 0x742
                    0x0742                  _OSCCON = 0x742
                    0x0742                  _OSCCONbits = 0x742
                    0x0742                  OSCCONL = 0x742
                    0x0742                  _OSCCONL = 0x742
                    0x0743                  OSCCONH = 0x743
                    0x0743                  _OSCCONH = 0x743
                    0x0744                  CLKDIV = 0x744
                    0x0744                  _CLKDIV = 0x744
                    0x0744                  _CLKDIVbits = 0x744
                    0x0748                  OSCTUN = 0x748
                    0x0748                  _OSCTUN = 0x748
                    0x0748                  _OSCTUNbits = 0x748
                    0x0760                  NVMCON = 0x760
                    0x0760                  _NVMCON = 0x760
                    0x0760                  _NVMCONbits = 0x760
                    0x0766                  NVMKEY = 0x766
                    0x0766                  _NVMKEY = 0x766
                    0x0770                  PMD1 = 0x770
                    0x0770                  _PMD1 = 0x770
                    0x0770                  _PMD1bits = 0x770
                    0x0772                  PMD2 = 0x772
                    0x0772                  _PMD2 = 0x772
                    0x0772                  _PMD2bits = 0x772
                    0x0774                  PMD3 = 0x774
                    0x0774                  _PMD3 = 0x774
                    0x0774                  _PMD3bits = 0x774
                    0x0140                  IC1 = 0x140
                    0x0140                  _IC1 = 0x140
                    0x0144                  IC2 = 0x144
                    0x0144                  _IC2 = 0x144
                    0x0148                  IC3 = 0x148
                    0x0148                  _IC3 = 0x148
                    0x014c                  IC4 = 0x14c
                    0x014c                  _IC4 = 0x14c
                    0x0150                  IC5 = 0x150
                    0x0150                  _IC5 = 0x150
                    0x0180                  OC1 = 0x180
                    0x0180                  _OC1 = 0x180
                    0x0186                  OC2 = 0x186
                    0x0186                  _OC2 = 0x186
                    0x018c                  OC3 = 0x18c
                    0x018c                  _OC3 = 0x18c
                    0x0192                  OC4 = 0x192
                    0x0192                  _OC4 = 0x192
                    0x0198                  OC5 = 0x198
                    0x0198                  _OC5 = 0x198
                    0x0240                  SPI1 = 0x240
                    0x0240                  _SPI1 = 0x240
                    0x0260                  SPI2 = 0x260
                    0x0260                  _SPI2 = 0x260
                    0x0220                  UART1 = 0x220
                    0x0220                  _UART1 = 0x220
                    0x0230                  UART2 = 0x230
                    0x0230                  _UART2 = 0x230
                    0x0001                  __MPLAB_BUILD = 0x1
START GROUP
LOAD c:/pic30_tools/bin/bin/../../lib\libpic30-coff.a
LOAD c:/pic30_tools/bin/bin/../../lib\libm-coff.a
LOAD c:/pic30_tools/bin/bin/../../lib\libc-coff.a
END GROUP
OUTPUT(COM4201_Lab2Solution-C30.cof coff-pic30)
LOAD data_init
LOAD default_isr

TCB_uRAM            0x0800        0x10e
 TCB_uRAM           0x0800        0x10e ..\Microchip\TCPIP Stack\Objects - COM4201Lab2Solution-C30\TCP.o

.nbss               0x090e        0x160
 .nbss              0x090e         0xc8 Objects - COM4201Lab2Solution-C30\CustomHTTPApp.o
 .nbss              0x09d6         0x98 ..\Microchip\TCPIP Stack\Objects - COM4201Lab2Solution-C30\UDP.o
                    0x09dc                  UDPSocketInfo
                    0x0a68                  activeUDPSocket
                    0x0a6a                  UDPTxCount
                    0x0a6c                  UDPRxCount

HTTP_CONNECTION_STATES
                    0x0a6e         0x8c
 HTTP_CONNECTION_STATES
                    0x0a6e         0x8c ..\Microchip\TCPIP Stack\Objects - COM4201Lab2Solution-C30\HTTP2.o
                    0x0a6e                  curHTTP
                    0x0af0                  httpStubs
                    0x0af8                  curHTTPID

.ndata              0x0afa         0x72
 .ndata             0x0afa         0x72 Objects - COM4201Lab2Solution-C30\BerkeleyTCPClientDemo.o

.nbss               0x0b6c         0xc4
 .nbss              0x0b6c         0x70 ..\Microchip\TCPIP Stack\Objects - COM4201Lab2Solution-C30\MPFS2.o
                    0x0bd8                  lastRead
 .nbss              0x0bdc         0x54 ..\Microchip\TCPIP Stack\Objects - COM4201Lab2Solution-C30\UART2TCPBridge.o

.ndata              0x0c30         0x50
 .ndata             0x0c30         0x50 ..\Microchip\TCPIP Stack\Objects - COM4201Lab2Solution-C30\HTTP2.o

.nbss               0x0c80         0x50
 .nbss              0x0c80         0x50 ..\Microchip\TCPIP Stack\Objects - COM4201Lab2Solution-C30\TCP.o

BSD_uRAM            0x0cd0         0x50
 BSD_uRAM           0x0cd0         0x50 ..\Microchip\TCPIP Stack\Objects - COM4201Lab2Solution-C30\BerkeleyAPI.o

.ndata              0x0d20         0x48
 .ndata             0x0d20         0x48 Objects - COM4201Lab2Solution-C30\SMTPDemo.o

.nbss               0x0d68         0x80
 .nbss              0x0d68         0x40 Objects - COM4201Lab2Solution-C30\MainDemo.o
                    0x0d6c                  AppConfig
                    0x0d9f                  AN0String
 .nbss              0x0da8         0x40 ..\Microchip\TCPIP Stack\Objects - COM4201Lab2Solution-C30\Hashes.o
                    0x0da8                  lastBlock

SYN_QUEUE_RAM_SECT
                    0x0de8         0x3c
 SYN_QUEUE_RAM_SECT
                    0x0de8         0x3c ..\Microchip\TCPIP Stack\Objects - COM4201Lab2Solution-C30\TCP.o

.nbss               0x0e24         0xe4
 .nbss              0x0e24         0x3a ..\Microchip\TCPIP Stack\Objects - COM4201Lab2Solution-C30\DynDNS.o
                    0x0e4e                  DDNSClient
 .nbss              0x0e5e         0x3a ..\Microchip\TCPIP Stack\Objects - COM4201Lab2Solution-C30\SMTP.o
                    0x0e80                  SMTPClient
 .nbss              0x0e98         0x28 Objects - COM4201Lab2Solution-C30\BerkeleyUDPClientDemo.o
 .nbss              0x0ec0         0x26 ..\Microchip\TCPIP Stack\Objects - COM4201Lab2Solution-C30\SPIEEPROM.o
 .nbss              0x0ee6         0x22 ..\Microchip\TCPIP Stack\Objects - COM4201Lab2Solution-C30\DHCP.o

.ndata              0x0f08         0x22
 .ndata             0x0f08         0x22 ..\Microchip\TCPIP Stack\Objects - COM4201Lab2Solution-C30\DynDNS.o
                    0x0f22                  ddnsServiceHosts

.nbss               0x0f2a         0xa2
 .nbss              0x0f2a         0x22 ..\Microchip\TCPIP Stack\Objects - COM4201Lab2Solution-C30\LCDBlocking.o
                    0x0f2a                  LCDText
 .nbss              0x0f4c         0x20 ..\Microchip\TCPIP Stack\Objects - COM4201Lab2Solution-C30\TCPPerformanceTest.o
 .nbss              0x0f6c         0x1a ..\Microchip\TCPIP Stack\Objects - COM4201Lab2Solution-C30\ICMP.o
 .nbss              0x0f86         0x1a ..\Microchip\TCPIP Stack\Objects - COM4201Lab2Solution-C30\SNTP.o
 .nbss              0x0fa0         0x16 ..\Microchip\TCPIP Stack\Objects - COM4201Lab2Solution-C30\ARP.o
 .nbss              0x0fb6         0x16 ..\Microchip\TCPIP Stack\Objects - COM4201Lab2Solution-C30\DNS.o

.ndata              0x0fcc         0x16
 .ndata             0x0fcc         0x16 Objects - COM4201Lab2Solution-C30\GenericTCPClient.o

.nbss               0x0fe2         0x44
 .nbss              0x0fe2         0x12 Objects - COM4201Lab2Solution-C30\BerkeleyTCPServerDemo.o
 .nbss              0x0ff4         0x10 Objects - COM4201Lab2Solution-C30\BerkeleyTCPClientDemo.o
 .nbss              0x1004          0xc ..\Microchip\TCPIP Stack\Objects - COM4201Lab2Solution-C30\StackTsk.o
                    0x1006                  remoteNode
 .nbss              0x1010          0xc ..\Microchip\TCPIP Stack\Objects - COM4201Lab2Solution-C30\BerkeleyAPI.o
 .nbss              0x101c          0xa ..\Microchip\TCPIP Stack\Objects - COM4201Lab2Solution-C30\Tick.o

.ndata              0x1026          0xa
 .ndata             0x1026          0xa ..\Microchip\TCPIP Stack\Objects - COM4201Lab2Solution-C30\UART2TCPBridge.o

.nbss               0x1030         0x10
 .nbss              0x1030          0x8 ..\Microchip\TCPIP Stack\Objects - COM4201Lab2Solution-C30\DHCPs.o
 .nbss              0x1038          0x8 ..\Microchip\TCPIP Stack\Objects - COM4201Lab2Solution-C30\ENC28J60.o

.ndata              0x1040          0x6
 .ndata             0x1040          0x6 ..\Microchip\TCPIP Stack\Objects - COM4201Lab2Solution-C30\DHCP.o
                    0x1040                  smDHCPState
                    0x1042                  DHCPFlags
                    0x1044                  DHCPBindCount

.nbss               0x1046         0x12
 .nbss              0x1046          0x6 ..\Microchip\TCPIP Stack\Objects - COM4201Lab2Solution-C30\Telnet.o
 .nbss              0x104c          0x6 Objects - COM4201Lab2Solution-C30\PingDemo.o
 .nbss              0x1052          0x6 Objects - COM4201Lab2Solution-C30\SMTPDemo.o

.ndata              0x1058          0x6
 .ndata             0x1058          0x6 Objects - COM4201Lab2Solution-C30\BerkeleyTCPServerDemo.o

.nbss               0x105e          0x4
 .nbss              0x105e          0x4 ..\Microchip\TCPIP Stack\Objects - COM4201Lab2Solution-C30\Announce.o

.ndata              0x1062          0x4
 .ndata             0x1062          0x4 ..\Microchip\TCPIP Stack\Objects - COM4201Lab2Solution-C30\DNS.o

.nbss               0x1066         0x10
 .nbss              0x1066          0x4 ..\Microchip\TCPIP Stack\Objects - COM4201Lab2Solution-C30\IP.o
 .nbss              0x106a          0x4 ..\Microchip\TCPIP Stack\Objects - COM4201Lab2Solution-C30\NBNS.o
 .nbss              0x106e          0x4 Objects - COM4201Lab2Solution-C30\GenericTCPClient.o
 .nbss              0x1072          0x4 Objects - COM4201Lab2Solution-C30\GenericTCPServer.o

.ndata              0x1076          0x8
 .ndata             0x1076          0x4 ..\Microchip\TCPIP Stack\Objects - COM4201Lab2Solution-C30\BerkeleyAPI.o
 .ndata             0x107a          0x2 Objects - COM4201Lab2Solution-C30\MainDemo.o
                    0x107a                  myDHCPBindCount
 .ndata             0x107c          0x2 ..\Microchip\TCPIP Stack\Objects - COM4201Lab2Solution-C30\UDP.o

_0145ba104acc9c92
                    0x107e          0x2
 _0145ba104acc9c92
                    0x107e          0x2 ..\Microchip\TCPIP Stack\Objects - COM4201Lab2Solution-C30\UDP.o

.ndata              0x1080          0x2
 .ndata             0x1080          0x2 ..\Microchip\TCPIP Stack\Objects - COM4201Lab2Solution-C30\DHCPs.o
                    0x1080                  bDHCPServerEnabled

_01478ee04acc9c98
                    0x1082          0x2
 _01478ee04acc9c98
                    0x1082          0x2 ..\Microchip\TCPIP Stack\Objects - COM4201Lab2Solution-C30\DNS.o

.ndata              0x1084          0x6
 .ndata             0x1084          0x2 ..\Microchip\TCPIP Stack\Objects - COM4201Lab2Solution-C30\Reboot.o
 .ndata             0x1086          0x2 ..\Microchip\TCPIP Stack\Objects - COM4201Lab2Solution-C30\SMTP.o
 .ndata             0x1088          0x2 ..\Microchip\TCPIP Stack\Objects - COM4201Lab2Solution-C30\TCP.o

_0148ca804acc9cab
                    0x108a          0x2
 _0148ca804acc9cab
                    0x108a          0x2 ..\Microchip\TCPIP Stack\Objects - COM4201Lab2Solution-C30\TCP.o

.ndata              0x108c          0x6
 .ndata             0x108c          0x2 ..\Microchip\TCPIP Stack\Objects - COM4201Lab2Solution-C30\TCPPerformanceTest.o
 .ndata             0x108e          0x2 ..\Microchip\TCPIP Stack\Objects - COM4201Lab2Solution-C30\Telnet.o
 .ndata             0x1090          0x2 Objects - COM4201Lab2Solution-C30\BerkeleyUDPClientDemo.o

.bss                0x1092         0x88
 .bss               0x1092         0x88 c:/pic30_tools/bin/bin/../../lib\libc-coff.a(rand.o)

.data               0x111a         0x58
 .data              0x111a         0x4a c:/pic30_tools/bin/bin/../../lib\libc-coff.a(xstoul.o)
 .data              0x1164          0xa c:/pic30_tools/bin/bin/../../lib\libc-coff.a(rand.o)
                    0x1164                  _Tls_setup__Randseed
                    0x1166                  _Randseed
                    0x116a                  _Tls_setup__Randinit
                    0x116c                  _Randinit
 .data              0x116e          0x4 c:/pic30_tools/bin/bin/../../lib\libc-coff.a(errno.o)
                    0x116e                  _Tls_setup_errno
                    0x1170                  errno

.const              0x8850       0x1658 load address 0x000850  
 .const             0x8850        0x714 ..\Microchip\TCPIP Stack\Objects - COM4201Lab2Solution-C30\HTTP2.o
 .const             0x8f64        0x48e Objects - COM4201Lab2Solution-C30\CustomHTTPApp.o
                    0x9249                  HTML_UP_ARROW
                    0x924c                  HTML_DOWN_ARROW
 .const             0x93f2        0x1fe Objects - COM4201Lab2Solution-C30\UARTConfig.o
 .const             0x95f0        0x1c2 ..\Microchip\TCPIP Stack\Objects - COM4201Lab2Solution-C30\Telnet.o
 .const             0x97b2        0x1a4 ..\Microchip\TCPIP Stack\Objects - COM4201Lab2Solution-C30\DynDNS.o
 .const             0x9956        0x140 ..\Microchip\TCPIP Stack\Objects - COM4201Lab2Solution-C30\Hashes.o
 .const             0x9a96        0x12e Objects - COM4201Lab2Solution-C30\BerkeleyTCPClientDemo.o
 .const             0x9bc4         0x8e Objects - COM4201Lab2Solution-C30\MainDemo.o
 .const             0x9c52         0x8e Objects - COM4201Lab2Solution-C30\GenericTCPClient.o
 .const             0x9ce0         0x86 ..\Microchip\TCPIP Stack\Objects - COM4201Lab2Solution-C30\SMTP.o
 .const             0x9d66         0x58 ..\Microchip\TCPIP Stack\Objects - COM4201Lab2Solution-C30\TCPPerformanceTest.o
 .const             0x9dbe         0x4a Objects - COM4201Lab2Solution-C30\SMTPDemo.o
 .const             0x9e08         0x36 ..\Microchip\TCPIP Stack\Objects - COM4201Lab2Solution-C30\TCP.o
                    0x9e08                  TCPSocketInitializer
 .const             0x9e3e         0x1c ..\Microchip\TCPIP Stack\Objects - COM4201Lab2Solution-C30\Announce.o
 .const             0x9e5a         0x18 Objects - COM4201Lab2Solution-C30\PingDemo.o
 .const             0x9e72         0x12 ..\Microchip\TCPIP Stack\Objects - COM4201Lab2Solution-C30\Reboot.o
 .const             0x9e84          0xe ..\Microchip\TCPIP Stack\Objects - COM4201Lab2Solution-C30\SNTP.o
 .const             0x9e92          0xe Objects - COM4201Lab2Solution-C30\BerkeleyUDPClientDemo.o
 .const             0x9ea0          0x8 ..\Microchip\TCPIP Stack\Objects - COM4201Lab2Solution-C30\MPFS2.o

.text             0x001ea8       0x20ac
 .text            0x001ea8       0x20ac ..\Microchip\TCPIP Stack\Objects - COM4201Lab2Solution-C30\TCP.o
                  0x001f5a                  TCPInit
                  0x00200a                  TCPOpen
                  0x002150                  TCPWasReset
                  0x002174                  TCPIsConnected
                  0x002190                  TCPDisconnect
                  0x0021fe                  TCPGetRemoteInfo
                  0x002216                  TCPFlush
                  0x002232                  TCPIsPutReady
                  0x00227c                  TCPPut
                  0x002308                  TCPPutArray
                  0x0023d6                  TCPPutString
                  0x0023f4                  TCPGetTxFIFOFull
                  0x002412                  TCPDiscard
                  0x002430                  TCPIsGetReady
                  0x002462                  TCPGet
                  0x0024cc                  TCPGetArray
                  0x002588                  TCPGetRxFIFOFree
                  0x0025a4                  TCPFindArrayEx
                  0x002828                  TCPFindEx
                  0x002846                  TCPTick
                  0x002cb4                  TCPProcess
                  0x003d3a                  TCPAdjustFIFOSize

.text             0x003f54       0x18ee
 .text            0x003f54       0x18ee Objects - COM4201Lab2Solution-C30\CustomHTTPApp.o
                  0x003f54                  HTTPNeedsAuth
                  0x003f76                  HTTPCheckAuth
                  0x003fa4                  HTTPExecuteGet
                  0x0041ce                  HTTPExecutePost
                  0x004e2c                  HTTPPrint_builddate
                  0x004e6c                  HTTPPrint_version
                  0x004e88                  HTTPPrint_btn
                  0x004f08                  HTTPPrint_led
                  0x004fd8                  HTTPPrint_ledSelected
                  0x0050b2                  HTTPPrint_pot
                  0x0050d8                  HTTPPrint_lcdtext
                  0x0051bc                  HTTPPrint_hellomsg
                  0x0051fa                  HTTPPrint_cookiename
                  0x00523a                  HTTPPrint_uploadedmd5
                  0x005314                  HTTPPrintIP
                  0x005368                  HTTPPrint_config_hostname
                  0x005382                  HTTPPrint_config_dhcpchecked
                  0x0053a6                  HTTPPrint_config_ip
                  0x0053cc                  HTTPPrint_config_gw
                  0x0053f2                  HTTPPrint_config_subnet
                  0x005418                  HTTPPrint_config_dns1
                  0x00543e                  HTTPPrint_config_dns2
                  0x005464                  HTTPPrint_config_mac
                  0x005502                  HTTPPrint_reboot
                  0x00550a                  HTTPPrint_rebootaddr
                  0x005524                  HTTPPrint_ddns_user
                  0x00557c                  HTTPPrint_ddns_pass
                  0x0055d4                  HTTPPrint_ddns_host
                  0x00562c                  HTTPPrint_ddns_service
                  0x00566c                  HTTPPrint_ddns_status
                  0x0056d4                  HTTPPrint_ddns_status_msg
                  0x0057c6                  HTTPPrint_status_ok
                  0x005804                  HTTPPrint_status_fail

.text             0x005842       0x17dc
 .text            0x005842       0x17dc ..\Microchip\TCPIP Stack\Objects - COM4201Lab2Solution-C30\HTTP2.o
                  0x005842                  HTTPPrint
                  0x005862                  HTTPPrint_
                  0x00587c                  HTTPInit
                  0x0058ec                  HTTPServer
                  0x006a1c                  HTTPURLDecode
                  0x006ae2                  HTTPGetArg
                  0x006b2a                  HTTPReadPostName
                  0x006b52                  HTTPReadPostValue
                  0x006f56                  HTTPIncFile

.text             0x00701e        0xec0
 .text            0x00701e        0xec0 ..\Microchip\TCPIP Stack\Objects - COM4201Lab2Solution-C30\SMTP.o
                  0x00701e                  SMTPBeginUsage
                  0x007072                  SMTPEndUsage
                  0x0070ba                  SMTPTask
                  0x007c16                  SMTPSendMail
                  0x007c1e                  SMTPIsBusy
                  0x007c34                  SMTPIsPutReady
                  0x007c50                  SMTPPut
                  0x007cf0                  SMTPPutArray
                  0x007d2c                  SMTPPutString
                  0x007d62                  SMTPFlush
                  0x007d6e                  SMTPPutDone

.text             0x007ede        0xc2a
 .text            0x007ede        0xc2a ..\Microchip\TCPIP Stack\Objects - COM4201Lab2Solution-C30\ENC28J60.o
                  0x007ede                  MACInit
                  0x008002                  MACIsLinked
                  0x008016                  MACIsTxReady
                  0x00802e                  MACDiscardRx
                  0x008062                  MACGetFreeRxSize
                  0x0080ea                  MACGetHeader
                  0x0081cc                  MACPutHeader
                  0x008220                  MACFlush
                  0x00833c                  MACSetReadPtrInRx
                  0x00836a                  MACSetWritePtr
                  0x008398                  MACSetReadPtr
                  0x0083c6                  MACCalcRxChecksum
                  0x00841e                  CalcIPBufferChecksum
                  0x0084d2                  MACMemCopyAsync
                  0x008680                  MACIsMemCopyDone
                  0x008698                  MACGet
                  0x0086c2                  MACGetArray
                  0x00878a                  MACPut
                  0x0087bc                  MACPutArray
                  0x008932                  ReadPHYReg
                  0x008a3a                  WritePHYReg
                  0x008a8a                  MACPowerDown
                  0x008ab8                  MACPowerUp
                  0x008ad8                  SetCLKOUT
                  0x008aee                  GetCLKOUT

.text             0x008b08        0xad2
 .text            0x008b08        0xad2 ..\Microchip\TCPIP Stack\Objects - COM4201Lab2Solution-C30\MPFS2.o
                  0x008b08                  MPFSInit
                  0x008b3e                  MPFSOpen
                  0x008c8c                  MPFSOpenID
                  0x008d10                  MPFSClose
                  0x008d32                  MPFSGet
                  0x008e38                  MPFSGetArray
                  0x008f4c                  MPFSGetLong
                  0x008f6c                  MPFSSeek
                  0x009148                  MPFSFormat
                  0x0091e2                  MPFSPutArray
                  0x009286                  MPFSPutEnd
                  0x0092e2                  MPFSGetTimestamp
                  0x009330                  MPFSGetMicrotime
                  0x00937e                  MPFSGetFlags
                  0x0093c2                  MPFSGetSize
                  0x009410                  MPFSGetBytesRem
                  0x009458                  MPFSGetStartAddr
                  0x0094a8                  MPFSGetEndAddr
                  0x009502                  MPFSGetFilename
                  0x00956a                  MPFSGetPosition
                  0x00958a                  MPFSGetID

.text             0x0095da        0x964
 .text            0x0095da        0x964 ..\Microchip\TCPIP Stack\Objects - COM4201Lab2Solution-C30\DynDNS.o
                  0x0095da                  DDNSInit
                  0x00961c                  DDNSTask
                  0x009ef4                  DDNSForceUpdate
                  0x009f0a                  DDNSSetService
                  0x009f2a                  DDNSGetLastIP
                  0x009f36                  DDNSGetLastStatus

.text             0x009f3e        0x956
 .text            0x009f3e        0x956 ..\Microchip\TCPIP Stack\Objects - COM4201Lab2Solution-C30\Helpers.o
                  0x009f3e                  GenerateRandomDWORD
                  0x00a058                  StringToIPAddress
                  0x00a1d8                  Base64Decode
                  0x00a33e                  Base64Encode
                  0x00a49a                  uitoa
                  0x00a518                  ultoa
                  0x00a5c8                  hexatob
                  0x00a63e                  btohexa_high
                  0x00a666                  btohexa_low
                  0x00a68c                  stricmppgm2ram
                  0x00a724                  swaps
                  0x00a73e                  swapl
                  0x00a79c                  CalcIPChecksum
                  0x00a812                  strupr
                  0x00a84c                  FormatNetBIOSName

.text             0x00a894        0x92a
 .text            0x00a894        0x92a ..\Microchip\TCPIP Stack\Objects - COM4201Lab2Solution-C30\BerkeleyAPI.o
                  0x00a894                  BerkeleySocketInit
                  0x00a8d6                  socket
                  0x00a954                  bind
                  0x00a9c8                  listen
                  0x00aa14                  accept
                  0x00ab40                  connect
                  0x00ac7e                  send
                  0x00adc0                  sendto
                  0x00af02                  recv
                  0x00b04c                  recvfrom
                  0x00b106                  gethostname
                  0x00b16a                  closesocket

.text             0x00b1be        0x8c2
 .text            0x00b1be        0x8c2 ..\Microchip\TCPIP Stack\Objects - COM4201Lab2Solution-C30\DHCP.o
                  0x00b1be                  DHCPReset
                  0x00b1e0                  DHCPDisable
                  0x00b1fc                  DHCPEnable
                  0x00b214                  DHCPTask

.text             0x00ba80        0x602
 .text            0x00ba80        0x602 ..\Microchip\TCPIP Stack\Objects - COM4201Lab2Solution-C30\DNS.o
                  0x00ba80                  DNSBeginUsage
                  0x00ba9c                  DNSEndUsage
                  0x00bac2                  DNSResolve
                  0x00baf2                  DNSIsResolved

.text             0x00c082        0x52e
 .text            0x00c082        0x52e ..\Microchip\TCPIP Stack\Objects - COM4201Lab2Solution-C30\UDP.o
                  0x00c082                  UDPInit
                  0x00c09c                  UDPTask
                  0x00c0a6                  UDPOpen
                  0x00c134                  UDPClose
                  0x00c15e                  UDPSetTxBuffer
                  0x00c172                  UDPSetRxBuffer
                  0x00c186                  UDPIsPutReady
                  0x00c1bc                  UDPPut
                  0x00c1f0                  UDPPutArray
                  0x00c228                  UDPPutString
                  0x00c23e                  UDPFlush
                  0x00c314                  UDPIsGetReady
                  0x00c340                  UDPGet
                  0x00c376                  UDPGetArray
                  0x00c3c0                  UDPDiscard
                  0x00c3d8                  UDPProcess

.text             0x00c5b0        0x51a
 .text            0x00c5b0        0x51a ..\Microchip\TCPIP Stack\Objects - COM4201Lab2Solution-C30\DHCPs.o
                  0x00c5b0                  DHCPServerTask

.text             0x00caca        0x4c4
 .text            0x00caca        0x4c4 ..\Microchip\TCPIP Stack\Objects - COM4201Lab2Solution-C30\Hashes.o
                  0x00caca                  HashAddData
                  0x00cae6                  MD5Initialize
                  0x00cb22                  MD5AddData
                  0x00ce22                  MD5Calculate

.text             0x00cf8e        0x434
 .text            0x00cf8e        0x434 Objects - COM4201Lab2Solution-C30\MainDemo.o
                  0x00cf8e                  _AddressError
                  0x00cf98                  _StackError
                  0x00cfa2                  main
                  0x00d0e2                  DisplayIPValue
                  0x00d38a                  SaveAppConfig

.text             0x00d3c2        0x42c
 .text            0x00d3c2        0x42c ..\Microchip\TCPIP Stack\Objects - COM4201Lab2Solution-C30\Telnet.o
                  0x00d3c2                  TelnetTask

.text             0x00d7ee        0x3a8
 .text            0x00d7ee        0x3a8 ..\Microchip\TCPIP Stack\Objects - COM4201Lab2Solution-C30\ARP.o
                  0x00d868                  ARPInit
                  0x00d89e                  ARPProcess
                  0x00d99e                  ARPResolve
                  0x00da6a                  ARPIsResolved

.text             0x00db96        0x386
 .text            0x00db96        0x386 ..\Microchip\TCPIP Stack\Objects - COM4201Lab2Solution-C30\NBNS.o
                  0x00db96                  NBNSTask

.text             0x00df1c        0x2cc
 .text            0x00df1c        0x2cc ..\Microchip\TCPIP Stack\Objects - COM4201Lab2Solution-C30\SNTP.o
                  0x00df1c                  SNTPClient
                  0x00e190                  SNTPGetUTCSeconds

.text             0x00e1e8        0x2b2
 .text            0x00e1e8        0x2b2 ..\Microchip\TCPIP Stack\Objects - COM4201Lab2Solution-C30\TCPPerformanceTest.o
                  0x00e1e8                  TCPPerformanceTask
                  0x00e1f2                  TCPTXPerformanceTask
                  0x00e388                  TCPRXPerformanceTask

.dinit            0x00e49a        0x2ac
 .dinit           0x00e49a        0x2ac data_init

.text             0x00e746        0x29e
 .text            0x00e746        0x29e Objects - COM4201Lab2Solution-C30\BerkeleyUDPClientDemo.o
                  0x00e746                  BerkeleyUDPClientDemo
                  0x00e98c                  BerkeleySNTPGetUTCSeconds

.text             0x00e9e4        0x274
 .text            0x00e9e4        0x274 ..\Microchip\TCPIP Stack\Objects - COM4201Lab2Solution-C30\StackTsk.o
                  0x00e9e4                  StackInit
                  0x00ea20                  StackTask
                  0x00ec26                  StackApplications

.text             0x00ec58        0x262
 .text            0x00ec58        0x262 Objects - COM4201Lab2Solution-C30\UARTConfig.o
                  0x00ec58                  DoUARTConfig

.text             0x00eeba        0x23a
 .text            0x00eeba        0x23a ..\Microchip\TCPIP Stack\Objects - COM4201Lab2Solution-C30\SPIEEPROM.o
                  0x00eeba                  XEEInit
                  0x00eed8                  XEEBeginRead
                  0x00eeec                  XEERead
                  0x00ef20                  XEEEndRead
                  0x00ef28                  XEEReadArray
                  0x00efb6                  XEEBeginWrite
                  0x00efca                  XEEWrite
                  0x00efe6                  XEEEndWrite
                  0x00f0b4                  XEEIsBusy

.text             0x00f0f4        0x234
 .text            0x00f0f4        0x234 ..\Microchip\TCPIP Stack\Objects - COM4201Lab2Solution-C30\ICMP.o
                  0x00f0f4                  ICMPProcess
                  0x00f1b6                  ICMPSendPing
                  0x00f234                  ICMPGetReply
                  0x00f304                  ICMPBeginUsage
                  0x00f320                  ICMPEndUsage

.text             0x00f328        0x1e0
 .text            0x00f328        0x1e0 ..\Microchip\TCPIP Stack\Objects - COM4201Lab2Solution-C30\UART2TCPBridge.o
                  0x00f328                  UART2TCPBridgeInit
                  0x00f33e                  UART2TCPBridgeTask
                  0x00f49a                  _U2RXInterrupt
                  0x00f4d8                  _U2TXInterrupt

.text             0x00f508        0x1ac
 .text            0x00f508        0x1ac ..\Microchip\TCPIP Stack\Objects - COM4201Lab2Solution-C30\IP.o
                  0x00f508                  IPGetHeader
                  0x00f5d2                  IPPutHeader
                  0x00f670                  IPSetRxBuffer

.text             0x00f6b4        0x1a8
 .text            0x00f6b4        0x1a8 ..\Microchip\TCPIP Stack\Objects - COM4201Lab2Solution-C30\LCDBlocking.o
                  0x00f6f8                  LCDInit
                  0x00f784                  LCDUpdate
                  0x00f840                  LCDErase

.text             0x00f85c        0x166
 .text            0x00f85c        0x166 ..\Microchip\TCPIP Stack\Objects - COM4201Lab2Solution-C30\Announce.o
                  0x00f85c                  AnnounceIP
                  0x00f8de                  DiscoveryTask

.text             0x00f9c2        0x15a
 .text            0x00f9c2        0x15a Objects - COM4201Lab2Solution-C30\GenericTCPClient.o
                  0x00f9c2                  GenericTCPClient

.text             0x00fb1c        0x152
 .text            0x00fb1c        0x152 ..\Microchip\TCPIP Stack\Objects - COM4201Lab2Solution-C30\UART.o
                  0x00fb1c                  ReadStringUART
                  0x00fb64                  putsUART2
                  0x00fbb2                  getsUART2
                  0x00fc1a                  DataRdyUART2
                  0x00fc26                  BusyUART2
                  0x00fc34                  ReadUART2
                  0x00fc52                  WriteUART2

.text             0x00fc6e        0x14e
 .text            0x00fc6e        0x14e ..\Microchip\TCPIP Stack\Objects - COM4201Lab2Solution-C30\Reboot.o
                  0x00fc6e                  RebootTask

.text             0x00fdbc        0x138
 .text            0x00fdbc        0x138 Objects - COM4201Lab2Solution-C30\BerkeleyTCPServerDemo.o
                  0x00fdbc                  BerkeleyTCPServerDemo

.text             0x00fef4        0x126
 .text            0x00fef4        0x126 Objects - COM4201Lab2Solution-C30\BerkeleyTCPClientDemo.o
                  0x00fef4                  BerkeleyTCPClientDemo

.text             0x01001a        0x106
 .text            0x01001a        0x106 Objects - COM4201Lab2Solution-C30\SMTPDemo.o
                  0x01001a                  SMTPDemo

.text             0x010120         0xfa
 .text            0x010120         0xfa ..\Microchip\TCPIP Stack\Objects - COM4201Lab2Solution-C30\Tick.o
                  0x010120                  TickInit
                  0x01019c                  TickGet
                  0x0101a8                  TickGetDiv256
                  0x0101c2                  TickGetDiv64K
                  0x0101dc                  TickConvertToMilliseconds
                  0x010202                  _T1Interrupt

.text             0x01021a         0xdc
 .text            0x01021a         0xdc Objects - COM4201Lab2Solution-C30\PingDemo.o
                  0x01021a                  PingDemo

.text             0x0102f6         0xd0
 .text            0x0102f6         0xd0 Objects - COM4201Lab2Solution-C30\GenericTCPServer.o
                  0x0102f6                  GenericTCPServer

.text             0x0103c6         0x56
 .text            0x0103c6         0x56 ..\Microchip\TCPIP Stack\Objects - COM4201Lab2Solution-C30\Delay.o
                  0x0103c6                  DelayMs
                  0x0103f0                  Delay10us

.isr              0x01041c          0x2
 .isr             0x01041c          0x2 default_isr
                  0x01041c                  _DefaultInterrupt
